 Iex_dll_d

 Timestamp is 44d97e42 (Tue Aug 08 23:18:42 2006)

 Preferred load address is 10000000

 Start         Length     Name                   Class
 0001:00000000 00010000H .textbss                DATA
 0002:00000000 0000907fH .text                   CODE
 0002:00009080 000010caH .text$x                 CODE
 0003:00000000 00000104H .CRT$XCA                DATA
 0003:00000104 00000104H .CRT$XCZ                DATA
 0003:00000208 00000104H .CRT$XIA                DATA
 0003:0000030c 00000104H .CRT$XIAA               DATA
 0003:00000410 00000104H .CRT$XIZ                DATA
 0003:00000520 00000e6bH .rdata                  DATA
 0003:0000138c 00000154H .rdata$debug            DATA
 0003:000014e0 00001662H .rdata$r                DATA
 0003:00002b44 00000104H .rtc$IAA                DATA
 0003:00002c48 00000109H .rtc$IMZ                DATA
 0003:00002d54 00000104H .rtc$IZZ                DATA
 0003:00002e58 00000104H .rtc$TAA                DATA
 0003:00002f5c 00000109H .rtc$TMZ                DATA
 0003:00003068 00000104H .rtc$TZZ                DATA
 0003:00003170 00001334H .xdata$x                DATA
 0003:000044a4 00000000H .edata                  DATA
 0004:00000000 00000833H .data                   DATA
 0004:00000838 0000043cH .bss                    DATA
 0005:00000000 0000003cH .idata$2                DATA
 0005:0000003c 00000014H .idata$3                DATA
 0005:00000050 000001d0H .idata$4                DATA
 0005:00000220 000001d0H .idata$5                DATA
 0005:000003f0 00000a08H .idata$6                DATA

  Address         Publics by Value              Rva+Base       Lib:Object

 0000:00000000       ___safe_se_handler_table   00000000     <absolute>
 0000:00000000       ___safe_se_handler_count   00000000     <absolute>
 0000:00000000       ___ImageBase               10000000     <linker-defined>
 0001:00000000       __enc$textbss$begin        10001000     <linker-defined>
 0001:00010000       __enc$textbss$end          10011000     <linker-defined>
 0002:00000c80       ?setStackTracer@Iex@@YAXP6A?AV?$basic_string@DU?$char_traits@D@std@@V?$allocator@D@2@@std@@XZ@Z 10011c80 f   IexBaseExc.obj
 0002:00000cc0       ?stackTracer@Iex@@YAP6A?AV?$basic_string@DU?$char_traits@D@std@@V?$allocator@D@2@@std@@XZXZ 10011cc0 f   IexBaseExc.obj
 0002:00000d00       ??0BaseExc@Iex@@QAE@PBD@Z  10011d00 f   IexBaseExc.obj
 0002:00000ec0       ??_GBaseExc@Iex@@UAEPAXI@Z 10011ec0 f i IexBaseExc.obj
 0002:00000ec0       ??_EBaseExc@Iex@@UAEPAXI@Z 10011ec0 f i IexBaseExc.obj
 0002:00000f30       ??0BaseExc@Iex@@QAE@ABV?$basic_string@DU?$char_traits@D@std@@V?$allocator@D@2@@std@@@Z 10011f30 f   IexBaseExc.obj
 0002:000010d0       ??0BaseExc@Iex@@QAE@AAV?$basic_stringstream@DU?$char_traits@D@std@@V?$allocator@D@2@@std@@@Z 100120d0 f   IexBaseExc.obj
 0002:00001270       ??0BaseExc@Iex@@QAE@ABV01@@Z 10012270 f   IexBaseExc.obj
 0002:00001350       ??1BaseExc@Iex@@UAE@XZ     10012350 f   IexBaseExc.obj
 0002:00001410       ?what@BaseExc@Iex@@UBEPBDXZ 10012410 f   IexBaseExc.obj
 0002:00001470       ?assign@BaseExc@Iex@@QAEAAV12@AAV?$basic_stringstream@DU?$char_traits@D@std@@V?$allocator@D@2@@std@@@Z 10012470 f   IexBaseExc.obj
 0002:00001580       ?append@BaseExc@Iex@@QAEAAV12@AAV?$basic_stringstream@DU?$char_traits@D@std@@V?$allocator@D@2@@std@@@Z 10012580 f   IexBaseExc.obj
 0002:00001690       ?throwErrnoExc@Iex@@YAXABV?$basic_string@DU?$char_traits@D@std@@V?$allocator@D@2@@std@@H@Z 10012690 f   IexThrowErrnoExc.obj
 0002:00001f40       ??0ErrnoExc@Iex@@QAE@ABV?$basic_string@DU?$char_traits@D@std@@V?$allocator@D@2@@std@@@Z 10012f40 f i IexThrowErrnoExc.obj
 0002:00001fb0       ??_EErrnoExc@Iex@@UAEPAXI@Z 10012fb0 f i IexThrowErrnoExc.obj
 0002:00001fb0       ??_GErrnoExc@Iex@@UAEPAXI@Z 10012fb0 f i IexThrowErrnoExc.obj
 0002:00002020       ??1ErrnoExc@Iex@@UAE@XZ    10013020 f i IexThrowErrnoExc.obj
 0002:00002070       ??0EpermExc@Iex@@QAE@ABV?$basic_string@DU?$char_traits@D@std@@V?$allocator@D@2@@std@@@Z 10013070 f i IexThrowErrnoExc.obj
 0002:000020e0       ??_GEpermExc@Iex@@UAEPAXI@Z 100130e0 f i IexThrowErrnoExc.obj
 0002:000020e0       ??_EEpermExc@Iex@@UAEPAXI@Z 100130e0 f i IexThrowErrnoExc.obj
 0002:00002150       ??1EpermExc@Iex@@UAE@XZ    10013150 f i IexThrowErrnoExc.obj
 0002:000021a0       ??0EnoentExc@Iex@@QAE@ABV?$basic_string@DU?$char_traits@D@std@@V?$allocator@D@2@@std@@@Z 100131a0 f i IexThrowErrnoExc.obj
 0002:00002210       ??_GEnoentExc@Iex@@UAEPAXI@Z 10013210 f i IexThrowErrnoExc.obj
 0002:00002210       ??_EEnoentExc@Iex@@UAEPAXI@Z 10013210 f i IexThrowErrnoExc.obj
 0002:00002280       ??1EnoentExc@Iex@@UAE@XZ   10013280 f i IexThrowErrnoExc.obj
 0002:000022d0       ??0EsrchExc@Iex@@QAE@ABV?$basic_string@DU?$char_traits@D@std@@V?$allocator@D@2@@std@@@Z 100132d0 f i IexThrowErrnoExc.obj
 0002:00002340       ??_GEsrchExc@Iex@@UAEPAXI@Z 10013340 f i IexThrowErrnoExc.obj
 0002:00002340       ??_EEsrchExc@Iex@@UAEPAXI@Z 10013340 f i IexThrowErrnoExc.obj
 0002:000023b0       ??1EsrchExc@Iex@@UAE@XZ    100133b0 f i IexThrowErrnoExc.obj
 0002:00002400       ??0EintrExc@Iex@@QAE@ABV?$basic_string@DU?$char_traits@D@std@@V?$allocator@D@2@@std@@@Z 10013400 f i IexThrowErrnoExc.obj
 0002:00002470       ??_GEintrExc@Iex@@UAEPAXI@Z 10013470 f i IexThrowErrnoExc.obj
 0002:00002470       ??_EEintrExc@Iex@@UAEPAXI@Z 10013470 f i IexThrowErrnoExc.obj
 0002:000024e0       ??1EintrExc@Iex@@UAE@XZ    100134e0 f i IexThrowErrnoExc.obj
 0002:00002530       ??0EioExc@Iex@@QAE@ABV?$basic_string@DU?$char_traits@D@std@@V?$allocator@D@2@@std@@@Z 10013530 f i IexThrowErrnoExc.obj
 0002:000025a0       ??_EEioExc@Iex@@UAEPAXI@Z  100135a0 f i IexThrowErrnoExc.obj
 0002:000025a0       ??_GEioExc@Iex@@UAEPAXI@Z  100135a0 f i IexThrowErrnoExc.obj
 0002:00002610       ??1EioExc@Iex@@UAE@XZ      10013610 f i IexThrowErrnoExc.obj
 0002:00002660       ??0EnxioExc@Iex@@QAE@ABV?$basic_string@DU?$char_traits@D@std@@V?$allocator@D@2@@std@@@Z 10013660 f i IexThrowErrnoExc.obj
 0002:000026d0       ??_EEnxioExc@Iex@@UAEPAXI@Z 100136d0 f i IexThrowErrnoExc.obj
 0002:000026d0       ??_GEnxioExc@Iex@@UAEPAXI@Z 100136d0 f i IexThrowErrnoExc.obj
 0002:00002740       ??1EnxioExc@Iex@@UAE@XZ    10013740 f i IexThrowErrnoExc.obj
 0002:00002790       ??0E2bigExc@Iex@@QAE@ABV?$basic_string@DU?$char_traits@D@std@@V?$allocator@D@2@@std@@@Z 10013790 f i IexThrowErrnoExc.obj
 0002:00002800       ??_EE2bigExc@Iex@@UAEPAXI@Z 10013800 f i IexThrowErrnoExc.obj
 0002:00002800       ??_GE2bigExc@Iex@@UAEPAXI@Z 10013800 f i IexThrowErrnoExc.obj
 0002:00002870       ??1E2bigExc@Iex@@UAE@XZ    10013870 f i IexThrowErrnoExc.obj
 0002:000028c0       ??0EnoexecExc@Iex@@QAE@ABV?$basic_string@DU?$char_traits@D@std@@V?$allocator@D@2@@std@@@Z 100138c0 f i IexThrowErrnoExc.obj
 0002:00002930       ??_EEnoexecExc@Iex@@UAEPAXI@Z 10013930 f i IexThrowErrnoExc.obj
 0002:00002930       ??_GEnoexecExc@Iex@@UAEPAXI@Z 10013930 f i IexThrowErrnoExc.obj
 0002:000029a0       ??1EnoexecExc@Iex@@UAE@XZ  100139a0 f i IexThrowErrnoExc.obj
 0002:000029f0       ??0EbadfExc@Iex@@QAE@ABV?$basic_string@DU?$char_traits@D@std@@V?$allocator@D@2@@std@@@Z 100139f0 f i IexThrowErrnoExc.obj
 0002:00002a60       ??_GEbadfExc@Iex@@UAEPAXI@Z 10013a60 f i IexThrowErrnoExc.obj
 0002:00002a60       ??_EEbadfExc@Iex@@UAEPAXI@Z 10013a60 f i IexThrowErrnoExc.obj
 0002:00002ad0       ??1EbadfExc@Iex@@UAE@XZ    10013ad0 f i IexThrowErrnoExc.obj
 0002:00002b20       ??0EchildExc@Iex@@QAE@ABV?$basic_string@DU?$char_traits@D@std@@V?$allocator@D@2@@std@@@Z 10013b20 f i IexThrowErrnoExc.obj
 0002:00002b90       ??_GEchildExc@Iex@@UAEPAXI@Z 10013b90 f i IexThrowErrnoExc.obj
 0002:00002b90       ??_EEchildExc@Iex@@UAEPAXI@Z 10013b90 f i IexThrowErrnoExc.obj
 0002:00002c00       ??1EchildExc@Iex@@UAE@XZ   10013c00 f i IexThrowErrnoExc.obj
 0002:00002c50       ??0EagainExc@Iex@@QAE@ABV?$basic_string@DU?$char_traits@D@std@@V?$allocator@D@2@@std@@@Z 10013c50 f i IexThrowErrnoExc.obj
 0002:00002cc0       ??_EEagainExc@Iex@@UAEPAXI@Z 10013cc0 f i IexThrowErrnoExc.obj
 0002:00002cc0       ??_GEagainExc@Iex@@UAEPAXI@Z 10013cc0 f i IexThrowErrnoExc.obj
 0002:00002d30       ??1EagainExc@Iex@@UAE@XZ   10013d30 f i IexThrowErrnoExc.obj
 0002:00002d80       ??0EnomemExc@Iex@@QAE@ABV?$basic_string@DU?$char_traits@D@std@@V?$allocator@D@2@@std@@@Z 10013d80 f i IexThrowErrnoExc.obj
 0002:00002df0       ??_GEnomemExc@Iex@@UAEPAXI@Z 10013df0 f i IexThrowErrnoExc.obj
 0002:00002df0       ??_EEnomemExc@Iex@@UAEPAXI@Z 10013df0 f i IexThrowErrnoExc.obj
 0002:00002e60       ??1EnomemExc@Iex@@UAE@XZ   10013e60 f i IexThrowErrnoExc.obj
 0002:00002eb0       ??0EaccesExc@Iex@@QAE@ABV?$basic_string@DU?$char_traits@D@std@@V?$allocator@D@2@@std@@@Z 10013eb0 f i IexThrowErrnoExc.obj
 0002:00002f20       ??_GEaccesExc@Iex@@UAEPAXI@Z 10013f20 f i IexThrowErrnoExc.obj
 0002:00002f20       ??_EEaccesExc@Iex@@UAEPAXI@Z 10013f20 f i IexThrowErrnoExc.obj
 0002:00002f90       ??1EaccesExc@Iex@@UAE@XZ   10013f90 f i IexThrowErrnoExc.obj
 0002:00002fe0       ??0EfaultExc@Iex@@QAE@ABV?$basic_string@DU?$char_traits@D@std@@V?$allocator@D@2@@std@@@Z 10013fe0 f i IexThrowErrnoExc.obj
 0002:00003050       ??_EEfaultExc@Iex@@UAEPAXI@Z 10014050 f i IexThrowErrnoExc.obj
 0002:00003050       ??_GEfaultExc@Iex@@UAEPAXI@Z 10014050 f i IexThrowErrnoExc.obj
 0002:000030c0       ??1EfaultExc@Iex@@UAE@XZ   100140c0 f i IexThrowErrnoExc.obj
 0002:00003110       ??0EbusyExc@Iex@@QAE@ABV?$basic_string@DU?$char_traits@D@std@@V?$allocator@D@2@@std@@@Z 10014110 f i IexThrowErrnoExc.obj
 0002:00003180       ??_EEbusyExc@Iex@@UAEPAXI@Z 10014180 f i IexThrowErrnoExc.obj
 0002:00003180       ??_GEbusyExc@Iex@@UAEPAXI@Z 10014180 f i IexThrowErrnoExc.obj
 0002:000031f0       ??1EbusyExc@Iex@@UAE@XZ    100141f0 f i IexThrowErrnoExc.obj
 0002:00003240       ??0EexistExc@Iex@@QAE@ABV?$basic_string@DU?$char_traits@D@std@@V?$allocator@D@2@@std@@@Z 10014240 f i IexThrowErrnoExc.obj
 0002:000032b0       ??_EEexistExc@Iex@@UAEPAXI@Z 100142b0 f i IexThrowErrnoExc.obj
 0002:000032b0       ??_GEexistExc@Iex@@UAEPAXI@Z 100142b0 f i IexThrowErrnoExc.obj
 0002:00003320       ??1EexistExc@Iex@@UAE@XZ   10014320 f i IexThrowErrnoExc.obj
 0002:00003370       ??0ExdevExc@Iex@@QAE@ABV?$basic_string@DU?$char_traits@D@std@@V?$allocator@D@2@@std@@@Z 10014370 f i IexThrowErrnoExc.obj
 0002:000033e0       ??_GExdevExc@Iex@@UAEPAXI@Z 100143e0 f i IexThrowErrnoExc.obj
 0002:000033e0       ??_EExdevExc@Iex@@UAEPAXI@Z 100143e0 f i IexThrowErrnoExc.obj
 0002:00003450       ??1ExdevExc@Iex@@UAE@XZ    10014450 f i IexThrowErrnoExc.obj
 0002:000034a0       ??0EnodevExc@Iex@@QAE@ABV?$basic_string@DU?$char_traits@D@std@@V?$allocator@D@2@@std@@@Z 100144a0 f i IexThrowErrnoExc.obj
 0002:00003510       ??_EEnodevExc@Iex@@UAEPAXI@Z 10014510 f i IexThrowErrnoExc.obj
 0002:00003510       ??_GEnodevExc@Iex@@UAEPAXI@Z 10014510 f i IexThrowErrnoExc.obj
 0002:00003580       ??1EnodevExc@Iex@@UAE@XZ   10014580 f i IexThrowErrnoExc.obj
 0002:000035d0       ??0EnotdirExc@Iex@@QAE@ABV?$basic_string@DU?$char_traits@D@std@@V?$allocator@D@2@@std@@@Z 100145d0 f i IexThrowErrnoExc.obj
 0002:00003640       ??_EEnotdirExc@Iex@@UAEPAXI@Z 10014640 f i IexThrowErrnoExc.obj
 0002:00003640       ??_GEnotdirExc@Iex@@UAEPAXI@Z 10014640 f i IexThrowErrnoExc.obj
 0002:000036b0       ??1EnotdirExc@Iex@@UAE@XZ  100146b0 f i IexThrowErrnoExc.obj
 0002:00003700       ??0EisdirExc@Iex@@QAE@ABV?$basic_string@DU?$char_traits@D@std@@V?$allocator@D@2@@std@@@Z 10014700 f i IexThrowErrnoExc.obj
 0002:00003770       ??_EEisdirExc@Iex@@UAEPAXI@Z 10014770 f i IexThrowErrnoExc.obj
 0002:00003770       ??_GEisdirExc@Iex@@UAEPAXI@Z 10014770 f i IexThrowErrnoExc.obj
 0002:000037e0       ??1EisdirExc@Iex@@UAE@XZ   100147e0 f i IexThrowErrnoExc.obj
 0002:00003830       ??0EinvalExc@Iex@@QAE@ABV?$basic_string@DU?$char_traits@D@std@@V?$allocator@D@2@@std@@@Z 10014830 f i IexThrowErrnoExc.obj
 0002:000038a0       ??_GEinvalExc@Iex@@UAEPAXI@Z 100148a0 f i IexThrowErrnoExc.obj
 0002:000038a0       ??_EEinvalExc@Iex@@UAEPAXI@Z 100148a0 f i IexThrowErrnoExc.obj
 0002:00003910       ??1EinvalExc@Iex@@UAE@XZ   10014910 f i IexThrowErrnoExc.obj
 0002:00003960       ??0EnfileExc@Iex@@QAE@ABV?$basic_string@DU?$char_traits@D@std@@V?$allocator@D@2@@std@@@Z 10014960 f i IexThrowErrnoExc.obj
 0002:000039d0       ??_GEnfileExc@Iex@@UAEPAXI@Z 100149d0 f i IexThrowErrnoExc.obj
 0002:000039d0       ??_EEnfileExc@Iex@@UAEPAXI@Z 100149d0 f i IexThrowErrnoExc.obj
 0002:00003a40       ??1EnfileExc@Iex@@UAE@XZ   10014a40 f i IexThrowErrnoExc.obj
 0002:00003a90       ??0EmfileExc@Iex@@QAE@ABV?$basic_string@DU?$char_traits@D@std@@V?$allocator@D@2@@std@@@Z 10014a90 f i IexThrowErrnoExc.obj
 0002:00003b00       ??_EEmfileExc@Iex@@UAEPAXI@Z 10014b00 f i IexThrowErrnoExc.obj
 0002:00003b00       ??_GEmfileExc@Iex@@UAEPAXI@Z 10014b00 f i IexThrowErrnoExc.obj
 0002:00003b70       ??1EmfileExc@Iex@@UAE@XZ   10014b70 f i IexThrowErrnoExc.obj
 0002:00003bc0       ??0EnottyExc@Iex@@QAE@ABV?$basic_string@DU?$char_traits@D@std@@V?$allocator@D@2@@std@@@Z 10014bc0 f i IexThrowErrnoExc.obj
 0002:00003c30       ??_GEnottyExc@Iex@@UAEPAXI@Z 10014c30 f i IexThrowErrnoExc.obj
 0002:00003c30       ??_EEnottyExc@Iex@@UAEPAXI@Z 10014c30 f i IexThrowErrnoExc.obj
 0002:00003ca0       ??1EnottyExc@Iex@@UAE@XZ   10014ca0 f i IexThrowErrnoExc.obj
 0002:00003cf0       ??0EfbigExc@Iex@@QAE@ABV?$basic_string@DU?$char_traits@D@std@@V?$allocator@D@2@@std@@@Z 10014cf0 f i IexThrowErrnoExc.obj
 0002:00003d60       ??_GEfbigExc@Iex@@UAEPAXI@Z 10014d60 f i IexThrowErrnoExc.obj
 0002:00003d60       ??_EEfbigExc@Iex@@UAEPAXI@Z 10014d60 f i IexThrowErrnoExc.obj
 0002:00003dd0       ??1EfbigExc@Iex@@UAE@XZ    10014dd0 f i IexThrowErrnoExc.obj
 0002:00003e20       ??0EnospcExc@Iex@@QAE@ABV?$basic_string@DU?$char_traits@D@std@@V?$allocator@D@2@@std@@@Z 10014e20 f i IexThrowErrnoExc.obj
 0002:00003e90       ??_EEnospcExc@Iex@@UAEPAXI@Z 10014e90 f i IexThrowErrnoExc.obj
 0002:00003e90       ??_GEnospcExc@Iex@@UAEPAXI@Z 10014e90 f i IexThrowErrnoExc.obj
 0002:00003f00       ??1EnospcExc@Iex@@UAE@XZ   10014f00 f i IexThrowErrnoExc.obj
 0002:00003f50       ??0EspipeExc@Iex@@QAE@ABV?$basic_string@DU?$char_traits@D@std@@V?$allocator@D@2@@std@@@Z 10014f50 f i IexThrowErrnoExc.obj
 0002:00003fc0       ??_GEspipeExc@Iex@@UAEPAXI@Z 10014fc0 f i IexThrowErrnoExc.obj
 0002:00003fc0       ??_EEspipeExc@Iex@@UAEPAXI@Z 10014fc0 f i IexThrowErrnoExc.obj
 0002:00004030       ??1EspipeExc@Iex@@UAE@XZ   10015030 f i IexThrowErrnoExc.obj
 0002:00004080       ??0ErofsExc@Iex@@QAE@ABV?$basic_string@DU?$char_traits@D@std@@V?$allocator@D@2@@std@@@Z 10015080 f i IexThrowErrnoExc.obj
 0002:000040f0       ??_EErofsExc@Iex@@UAEPAXI@Z 100150f0 f i IexThrowErrnoExc.obj
 0002:000040f0       ??_GErofsExc@Iex@@UAEPAXI@Z 100150f0 f i IexThrowErrnoExc.obj
 0002:00004160       ??1ErofsExc@Iex@@UAE@XZ    10015160 f i IexThrowErrnoExc.obj
 0002:000041b0       ??0EmlinkExc@Iex@@QAE@ABV?$basic_string@DU?$char_traits@D@std@@V?$allocator@D@2@@std@@@Z 100151b0 f i IexThrowErrnoExc.obj
 0002:00004220       ??_GEmlinkExc@Iex@@UAEPAXI@Z 10015220 f i IexThrowErrnoExc.obj
 0002:00004220       ??_EEmlinkExc@Iex@@UAEPAXI@Z 10015220 f i IexThrowErrnoExc.obj
 0002:00004290       ??1EmlinkExc@Iex@@UAE@XZ   10015290 f i IexThrowErrnoExc.obj
 0002:000042e0       ??0EpipeExc@Iex@@QAE@ABV?$basic_string@DU?$char_traits@D@std@@V?$allocator@D@2@@std@@@Z 100152e0 f i IexThrowErrnoExc.obj
 0002:00004350       ??_GEpipeExc@Iex@@UAEPAXI@Z 10015350 f i IexThrowErrnoExc.obj
 0002:00004350       ??_EEpipeExc@Iex@@UAEPAXI@Z 10015350 f i IexThrowErrnoExc.obj
 0002:000043c0       ??1EpipeExc@Iex@@UAE@XZ    100153c0 f i IexThrowErrnoExc.obj
 0002:00004410       ??0EdomExc@Iex@@QAE@ABV?$basic_string@DU?$char_traits@D@std@@V?$allocator@D@2@@std@@@Z 10015410 f i IexThrowErrnoExc.obj
 0002:00004480       ??_GEdomExc@Iex@@UAEPAXI@Z 10015480 f i IexThrowErrnoExc.obj
 0002:00004480       ??_EEdomExc@Iex@@UAEPAXI@Z 10015480 f i IexThrowErrnoExc.obj
 0002:000044f0       ??1EdomExc@Iex@@UAE@XZ     100154f0 f i IexThrowErrnoExc.obj
 0002:00004540       ??0ErangeExc@Iex@@QAE@ABV?$basic_string@DU?$char_traits@D@std@@V?$allocator@D@2@@std@@@Z 10015540 f i IexThrowErrnoExc.obj
 0002:000045b0       ??_EErangeExc@Iex@@UAEPAXI@Z 100155b0 f i IexThrowErrnoExc.obj
 0002:000045b0       ??_GErangeExc@Iex@@UAEPAXI@Z 100155b0 f i IexThrowErrnoExc.obj
 0002:00004620       ??1ErangeExc@Iex@@UAE@XZ   10015620 f i IexThrowErrnoExc.obj
 0002:00004670       ??0EdeadlkExc@Iex@@QAE@ABV?$basic_string@DU?$char_traits@D@std@@V?$allocator@D@2@@std@@@Z 10015670 f i IexThrowErrnoExc.obj
 0002:000046e0       ??_EEdeadlkExc@Iex@@UAEPAXI@Z 100156e0 f i IexThrowErrnoExc.obj
 0002:000046e0       ??_GEdeadlkExc@Iex@@UAEPAXI@Z 100156e0 f i IexThrowErrnoExc.obj
 0002:00004750       ??1EdeadlkExc@Iex@@UAE@XZ  10015750 f i IexThrowErrnoExc.obj
 0002:000047a0       ??0EnolckExc@Iex@@QAE@ABV?$basic_string@DU?$char_traits@D@std@@V?$allocator@D@2@@std@@@Z 100157a0 f i IexThrowErrnoExc.obj
 0002:00004810       ??_EEnolckExc@Iex@@UAEPAXI@Z 10015810 f i IexThrowErrnoExc.obj
 0002:00004810       ??_GEnolckExc@Iex@@UAEPAXI@Z 10015810 f i IexThrowErrnoExc.obj
 0002:00004880       ??1EnolckExc@Iex@@UAE@XZ   10015880 f i IexThrowErrnoExc.obj
 0002:000048d0       ??0EnametoolongExc@Iex@@QAE@ABV?$basic_string@DU?$char_traits@D@std@@V?$allocator@D@2@@std@@@Z 100158d0 f i IexThrowErrnoExc.obj
 0002:00004940       ??_GEnametoolongExc@Iex@@UAEPAXI@Z 10015940 f i IexThrowErrnoExc.obj
 0002:00004940       ??_EEnametoolongExc@Iex@@UAEPAXI@Z 10015940 f i IexThrowErrnoExc.obj
 0002:000049b0       ??1EnametoolongExc@Iex@@UAE@XZ 100159b0 f i IexThrowErrnoExc.obj
 0002:00004a00       ??0EilseqExc@Iex@@QAE@ABV?$basic_string@DU?$char_traits@D@std@@V?$allocator@D@2@@std@@@Z 10015a00 f i IexThrowErrnoExc.obj
 0002:00004a70       ??_EEilseqExc@Iex@@UAEPAXI@Z 10015a70 f i IexThrowErrnoExc.obj
 0002:00004a70       ??_GEilseqExc@Iex@@UAEPAXI@Z 10015a70 f i IexThrowErrnoExc.obj
 0002:00004ae0       ??1EilseqExc@Iex@@UAE@XZ   10015ae0 f i IexThrowErrnoExc.obj
 0002:00004b30       ??0EnosysExc@Iex@@QAE@ABV?$basic_string@DU?$char_traits@D@std@@V?$allocator@D@2@@std@@@Z 10015b30 f i IexThrowErrnoExc.obj
 0002:00004ba0       ??_GEnosysExc@Iex@@UAEPAXI@Z 10015ba0 f i IexThrowErrnoExc.obj
 0002:00004ba0       ??_EEnosysExc@Iex@@UAEPAXI@Z 10015ba0 f i IexThrowErrnoExc.obj
 0002:00004c10       ??1EnosysExc@Iex@@UAE@XZ   10015c10 f i IexThrowErrnoExc.obj
 0002:00004c60       ??0EnotemptyExc@Iex@@QAE@ABV?$basic_string@DU?$char_traits@D@std@@V?$allocator@D@2@@std@@@Z 10015c60 f i IexThrowErrnoExc.obj
 0002:00004cd0       ??_EEnotemptyExc@Iex@@UAEPAXI@Z 10015cd0 f i IexThrowErrnoExc.obj
 0002:00004cd0       ??_GEnotemptyExc@Iex@@UAEPAXI@Z 10015cd0 f i IexThrowErrnoExc.obj
 0002:00004d40       ??1EnotemptyExc@Iex@@UAE@XZ 10015d40 f i IexThrowErrnoExc.obj
 0002:00004d90       ??0EpermExc@Iex@@QAE@ABV01@@Z 10015d90 f i IexThrowErrnoExc.obj
 0002:00004e00       ??0ErrnoExc@Iex@@QAE@ABV01@@Z 10015e00 f i IexThrowErrnoExc.obj
 0002:00004e70       ??0EnoentExc@Iex@@QAE@ABV01@@Z 10015e70 f i IexThrowErrnoExc.obj
 0002:00004ee0       ??0EsrchExc@Iex@@QAE@ABV01@@Z 10015ee0 f i IexThrowErrnoExc.obj
 0002:00004f50       ??0EintrExc@Iex@@QAE@ABV01@@Z 10015f50 f i IexThrowErrnoExc.obj
 0002:00004fc0       ??0EioExc@Iex@@QAE@ABV01@@Z 10015fc0 f i IexThrowErrnoExc.obj
 0002:00005030       ??0EnxioExc@Iex@@QAE@ABV01@@Z 10016030 f i IexThrowErrnoExc.obj
 0002:000050a0       ??0E2bigExc@Iex@@QAE@ABV01@@Z 100160a0 f i IexThrowErrnoExc.obj
 0002:00005110       ??0EnoexecExc@Iex@@QAE@ABV01@@Z 10016110 f i IexThrowErrnoExc.obj
 0002:00005180       ??0EbadfExc@Iex@@QAE@ABV01@@Z 10016180 f i IexThrowErrnoExc.obj
 0002:000051f0       ??0EchildExc@Iex@@QAE@ABV01@@Z 100161f0 f i IexThrowErrnoExc.obj
 0002:00005260       ??0EagainExc@Iex@@QAE@ABV01@@Z 10016260 f i IexThrowErrnoExc.obj
 0002:000052d0       ??0EnomemExc@Iex@@QAE@ABV01@@Z 100162d0 f i IexThrowErrnoExc.obj
 0002:00005340       ??0EaccesExc@Iex@@QAE@ABV01@@Z 10016340 f i IexThrowErrnoExc.obj
 0002:000053b0       ??0EfaultExc@Iex@@QAE@ABV01@@Z 100163b0 f i IexThrowErrnoExc.obj
 0002:00005420       ??0EbusyExc@Iex@@QAE@ABV01@@Z 10016420 f i IexThrowErrnoExc.obj
 0002:00005490       ??0EexistExc@Iex@@QAE@ABV01@@Z 10016490 f i IexThrowErrnoExc.obj
 0002:00005500       ??0ExdevExc@Iex@@QAE@ABV01@@Z 10016500 f i IexThrowErrnoExc.obj
 0002:00005570       ??0EnodevExc@Iex@@QAE@ABV01@@Z 10016570 f i IexThrowErrnoExc.obj
 0002:000055e0       ??0EnotdirExc@Iex@@QAE@ABV01@@Z 100165e0 f i IexThrowErrnoExc.obj
 0002:00005650       ??0EisdirExc@Iex@@QAE@ABV01@@Z 10016650 f i IexThrowErrnoExc.obj
 0002:000056c0       ??0EinvalExc@Iex@@QAE@ABV01@@Z 100166c0 f i IexThrowErrnoExc.obj
 0002:00005730       ??0EnfileExc@Iex@@QAE@ABV01@@Z 10016730 f i IexThrowErrnoExc.obj
 0002:000057a0       ??0EmfileExc@Iex@@QAE@ABV01@@Z 100167a0 f i IexThrowErrnoExc.obj
 0002:00005810       ??0EnottyExc@Iex@@QAE@ABV01@@Z 10016810 f i IexThrowErrnoExc.obj
 0002:00005880       ??0EfbigExc@Iex@@QAE@ABV01@@Z 10016880 f i IexThrowErrnoExc.obj
 0002:000058f0       ??0EnospcExc@Iex@@QAE@ABV01@@Z 100168f0 f i IexThrowErrnoExc.obj
 0002:00005960       ??0EspipeExc@Iex@@QAE@ABV01@@Z 10016960 f i IexThrowErrnoExc.obj
 0002:000059d0       ??0ErofsExc@Iex@@QAE@ABV01@@Z 100169d0 f i IexThrowErrnoExc.obj
 0002:00005a40       ??0EmlinkExc@Iex@@QAE@ABV01@@Z 10016a40 f i IexThrowErrnoExc.obj
 0002:00005ab0       ??0EpipeExc@Iex@@QAE@ABV01@@Z 10016ab0 f i IexThrowErrnoExc.obj
 0002:00005b20       ??0EdomExc@Iex@@QAE@ABV01@@Z 10016b20 f i IexThrowErrnoExc.obj
 0002:00005b90       ??0ErangeExc@Iex@@QAE@ABV01@@Z 10016b90 f i IexThrowErrnoExc.obj
 0002:00005c00       ??0EdeadlkExc@Iex@@QAE@ABV01@@Z 10016c00 f i IexThrowErrnoExc.obj
 0002:00005c70       ??0EnolckExc@Iex@@QAE@ABV01@@Z 10016c70 f i IexThrowErrnoExc.obj
 0002:00005ce0       ??0EnametoolongExc@Iex@@QAE@ABV01@@Z 10016ce0 f i IexThrowErrnoExc.obj
 0002:00005d50       ??0EilseqExc@Iex@@QAE@ABV01@@Z 10016d50 f i IexThrowErrnoExc.obj
 0002:00005dc0       ??0EnosysExc@Iex@@QAE@ABV01@@Z 10016dc0 f i IexThrowErrnoExc.obj
 0002:00005e30       ??0EnotemptyExc@Iex@@QAE@ABV01@@Z 10016e30 f i IexThrowErrnoExc.obj
 0002:00005ea0       ?throwErrnoExc@Iex@@YAXABV?$basic_string@DU?$char_traits@D@std@@V?$allocator@D@2@@std@@@Z 10016ea0 f   IexThrowErrnoExc.obj
 0002:00005f04       ??1?$basic_string@DU?$char_traits@D@std@@V?$allocator@D@2@@std@@QAE@XZ 10016f04 f   msvcprtd:MSVCP80D.dll
 0002:00005f0a       ??0?$basic_string@DU?$char_traits@D@std@@V?$allocator@D@2@@std@@QAE@ABV01@@Z 10016f0a f   msvcprtd:MSVCP80D.dll
 0002:00005f10       ??0?$basic_string@DU?$char_traits@D@std@@V?$allocator@D@2@@std@@QAE@PBD@Z 10016f10 f   msvcprtd:MSVCP80D.dll
 0002:00005f16       ?str@?$basic_stringstream@DU?$char_traits@D@std@@V?$allocator@D@2@@std@@QBE?AV?$basic_string@DU?$char_traits@D@std@@V?$allocator@D@2@@2@XZ 10016f16 f   msvcprtd:MSVCP80D.dll
 0002:00005f1c       ?c_str@?$basic_string@DU?$char_traits@D@std@@V?$allocator@D@2@@std@@QBEPBDXZ 10016f1c f   msvcprtd:MSVCP80D.dll
 0002:00005f22       ?assign@?$basic_string@DU?$char_traits@D@std@@V?$allocator@D@2@@std@@QAEAAV12@ABV12@@Z 10016f22 f   msvcprtd:MSVCP80D.dll
 0002:00005f28       ?append@?$basic_string@DU?$char_traits@D@std@@V?$allocator@D@2@@std@@QAEAAV12@ABV12@@Z 10016f28 f   msvcprtd:MSVCP80D.dll
 0002:00005f2e       ?replace@?$basic_string@DU?$char_traits@D@std@@V?$allocator@D@2@@std@@QAEAAV12@IIPBDI@Z 10016f2e f   msvcprtd:MSVCP80D.dll
 0002:00005f34       ?find@?$basic_string@DU?$char_traits@D@std@@V?$allocator@D@2@@std@@QBEIPBDI@Z 10016f34 f   msvcprtd:MSVCP80D.dll
 0002:00005f3a       ??0?$_String_val@DV?$allocator@D@std@@@std@@QAE@ABV01@@Z 10016f3a f   msvcprtd:MSVCP80D.dll
 0002:00005f40       ??0_String_base@std@@QAE@ABV01@@Z 10016f40 f   msvcprtd:MSVCP80D.dll
 0002:00005f46       ??0_Container_base@std@@QAE@ABV01@@Z 10016f46 f   msvcprtd:MSVCP80D.dll
 0002:00005f50       __RTC_InitBase             10016f50 f   MSVCRTD:init.obj
 0002:00005f90       __RTC_Shutdown             10016f90 f   MSVCRTD:init.obj
 0002:00005fa8       ??0exception@std@@QAE@XZ   10016fa8 f   MSVCRTD:MSVCR80D.dll
 0002:00005fb0       __RTC_CheckEsp             10016fb0 f   MSVCRTD:stack.obj
 0002:00005fe0       @_RTC_CheckStackVars@8     10016fe0 f   MSVCRTD:stack.obj
 0002:00006060       @_RTC_AllocaHelper@12      10017060 f   MSVCRTD:stack.obj
 0002:000060a0       @_RTC_CheckStackVars2@12   100170a0 f   MSVCRTD:stack.obj
 0002:000061b0       ??0type_info@@AAE@ABV0@@Z  100171b0 f   MSVCRTD:ti_inst.obj
 0002:000061d0       ??_Etype_info@@UAEPAXI@Z   100171d0 f i MSVCRTD:ti_inst.obj
 0002:00006260       ??4type_info@@AAEAAV0@ABV0@@Z 10017260 f   MSVCRTD:ti_inst.obj
 0002:00006274       ??3@YAXPAX@Z               10017274 f   MSVCRTD:MSVCR80D.dll
 0002:0000627a       ??1exception@std@@UAE@XZ   1001727a f   MSVCRTD:MSVCR80D.dll
 0002:00006280       ___CxxFrameHandler3        10017280 f   MSVCRTD:MSVCR80D.dll
 0002:00006290       @__security_check_cookie@4 10017290 f   MSVCRTD:secchk.obj
 0002:000062a2       _strlen                    100172a2 f   MSVCRTD:MSVCR80D.dll
 0002:000062a8       _strerror                  100172a8 f   MSVCRTD:MSVCR80D.dll
 0002:000062ae       __CxxThrowException@8      100172ae f   MSVCRTD:MSVCR80D.dll
 0002:000062b4       ??0exception@std@@QAE@ABV01@@Z 100172b4 f   MSVCRTD:MSVCR80D.dll
 0002:000062ba       __errno                    100172ba f   MSVCRTD:MSVCR80D.dll
 0002:00006360       __CRT_INIT@12              10017360 f   MSVCRTD:crtdll.obj
 0002:00006620       _NtCurrentTeb              10017620 f i MSVCRTD:crtdll.obj
 0002:00006630       __DllMainCRTStartup@12     10017630 f   MSVCRTD:crtdll.obj
 0002:00006890       __RTC_NumErrors            10017890 f   MSVCRTD:userapi.obj
 0002:000068a0       __RTC_GetErrDesc           100178a0 f   MSVCRTD:userapi.obj
 0002:000068c0       __RTC_SetErrorType         100178c0 f   MSVCRTD:userapi.obj
 0002:000068f0       __RTC_SetErrorFunc         100178f0 f   MSVCRTD:userapi.obj
 0002:00006920       __RTC_SetErrorFuncW        10017920 f   MSVCRTD:userapi.obj
 0002:00006950       ?_RTC_GetErrorFunc@@YAP6AHHPBDH00ZZPBX@Z 10017950 f   MSVCRTD:userapi.obj
 0002:00006960       ?_RTC_GetErrorFuncW@@YAP6AHHPB_WH00ZZPBX@Z 10017960 f   MSVCRTD:userapi.obj
 0002:00006966       __CRT_RTC_INITW            10017966 f   MSVCRTD:MSVCR80D.dll
 0002:00006970       _DebuggerKnownHandle       10017970 f   MSVCRTD:error.obj
 0002:00006a40       ?_RTC_Failure@@YAXPAXH@Z   10017a40 f   MSVCRTD:error.obj
 0002:00006e40       ?_RTC_StackFailure@@YAXPAXPBD@Z 10017e40 f   MSVCRTD:error.obj
 0002:00006fb0       ?_RTC_AllocaFailure@@YAXPAXPAU_RTC_ALLOCA_NODE@@H@Z 10017fb0 f   MSVCRTD:error.obj
 0002:000071c0       __RTC_UninitUse            100181c0 f   MSVCRTD:error.obj
 0002:00007310       ??_M@YGXPAXIHP6EX0@Z@Z     10018310 f   MSVCRTD:ehvecdtr.obj
 0002:000073f0       ?__ArrayUnwind@@YGXPAXIHP6EX0@Z@Z 100183f0 f   MSVCRTD:ehvecdtr.obj
 0002:000074e0       ___report_gsfailure        100184e0 f   MSVCRTD:gs_report.obj
 0002:00007630       ___clean_type_info_names   10018630 f   MSVCRTD:tncleanup.obj
 0002:00007650       __onexit                   10018650 f   MSVCRTD:atonexit.obj
 0002:00007790       _atexit                    10018790 f   MSVCRTD:atonexit.obj
 0002:000077b0       __RTC_Initialize           100187b0 f   MSVCRTD:initsect.obj
 0002:000077e0       __RTC_Terminate            100187e0 f   MSVCRTD:initsect.obj
 0002:0000780e       __encode_pointer           1001880e f   MSVCRTD:MSVCR80D.dll
 0002:00007814       __malloc_dbg               10018814 f   MSVCRTD:MSVCR80D.dll
 0002:0000781a       __encoded_null             1001881a f   MSVCRTD:MSVCR80D.dll
 0002:00007820       __free_dbg                 10018820 f   MSVCRTD:MSVCR80D.dll
 0002:00007826       __decode_pointer           10018826 f   MSVCRTD:MSVCR80D.dll
 0002:0000782c       __CrtSetCheckCount         1001882c f   MSVCRTD:MSVCR80D.dll
 0002:00007840       __ValidateImageBase        10018840 f   MSVCRTD:pesect.obj
 0002:000078c0       __FindPESection            100188c0 f   MSVCRTD:pesect.obj
 0002:00007950       __IsNonwritableInCurrentImage 10018950 f   MSVCRTD:pesect.obj
 0002:00007aa4       __initterm                 10018aa4 f   MSVCRTD:MSVCR80D.dll
 0002:00007aaa       __initterm_e               10018aaa f   MSVCRTD:MSVCR80D.dll
 0002:00007ab0       __amsg_exit                10018ab0 f   MSVCRTD:MSVCR80D.dll
 0002:00007ac0       ___security_init_cookie    10018ac0 f   MSVCRTD:gs_support.obj
 0002:00007c20       ___CppXcptFilter           10018c20 f   MSVCRTD:MSVCR80D.dll
 0002:00007c30       _DllMain@12                10018c30 f   MSVCRTD:dllmain.obj
 0002:00007c60       __except_handler4          10018c60 f   MSVCRTD:chandler4gs.obj
 0002:00007c90       ?_RTC_GetSrcLine@@YAHPAEPA_WKPAH1K@Z 10018c90 f   MSVCRTD:pdblkup.obj
 0002:0000823c       ?terminate@@YAXXZ          1001923c f   MSVCRTD:MSVCR80D.dll
 0002:00008242       ??1type_info@@UAE@XZ       10019242 f   MSVCRTD:MSVCR80D.dll
 0002:00008242       ?_type_info_dtor_internal_method@type_info@@QAEXXZ 10019242 f   MSVCRTD:MSVCR80D.dll
 0002:00008248       __crt_debugger_hook        10019248 f   MSVCRTD:MSVCR80D.dll
 0002:0000824e       ___clean_type_info_names_internal 1001924e f   MSVCRTD:MSVCR80D.dll
 0002:00008254       __unlock                   10019254 f   MSVCRTD:MSVCR80D.dll
 0002:0000825a       ___dllonexit               1001925a f   MSVCRTD:MSVCR80D.dll
 0002:00008260       __lock                     10019260 f   MSVCRTD:MSVCR80D.dll
 0002:00008266       __except_handler4_common   10019266 f   MSVCRTD:MSVCR80D.dll
 0002:0000826c       _InterlockedExchange@8     1001926c f   kernel32:KERNEL32.dll
 0002:00008272       _Sleep@4                   10019272 f   kernel32:KERNEL32.dll
 0002:00008278       _InterlockedCompareExchange@12 10019278 f   kernel32:KERNEL32.dll
 0002:0000827e       _RaiseException@16         1001927e f   kernel32:KERNEL32.dll
 0002:00008284       _DebugBreak@0              10019284 f   kernel32:KERNEL32.dll
 0002:0000828a       _WideCharToMultiByte@32    1001928a f   kernel32:KERNEL32.dll
 0002:00008290       _IsDebuggerPresent@0       10019290 f   kernel32:KERNEL32.dll
 0002:00008296       _MultiByteToWideChar@24    10019296 f   kernel32:KERNEL32.dll
 0002:0000829c       _lstrlenA@4                1001929c f   kernel32:KERNEL32.dll
 0002:000082a2       _GetProcAddress@8          100192a2 f   kernel32:KERNEL32.dll
 0002:000082a8       _LoadLibraryA@4            100192a8 f   kernel32:KERNEL32.dll
 0002:000082ae       _TerminateProcess@8        100192ae f   kernel32:KERNEL32.dll
 0002:000082b4       _GetCurrentProcess@0       100192b4 f   kernel32:KERNEL32.dll
 0002:000082ba       _UnhandledExceptionFilter@4 100192ba f   kernel32:KERNEL32.dll
 0002:000082c0       _SetUnhandledExceptionFilter@4 100192c0 f   kernel32:KERNEL32.dll
 0002:000082c6       _QueryPerformanceCounter@4 100192c6 f   kernel32:KERNEL32.dll
 0002:000082cc       _GetTickCount@0            100192cc f   kernel32:KERNEL32.dll
 0002:000082d2       _GetCurrentThreadId@0      100192d2 f   kernel32:KERNEL32.dll
 0002:000082d8       _GetCurrentProcessId@0     100192d8 f   kernel32:KERNEL32.dll
 0002:000082de       _GetSystemTimeAsFileTime@4 100192de f   kernel32:KERNEL32.dll
 0002:000082e4       _FatalAppExitA@8           100192e4 f   kernel32:KERNEL32.dll
 0002:000082ea       _DisableThreadLibraryCalls@4 100192ea f   kernel32:KERNEL32.dll
 0002:000082f0       _HeapFree@12               100192f0 f   kernel32:KERNEL32.dll
 0002:000082f6       _HeapAlloc@12              100192f6 f   kernel32:KERNEL32.dll
 0002:000082fc       _GetProcessHeap@0          100192fc f   kernel32:KERNEL32.dll
 0002:00008302       _GetModuleFileNameW@12     10019302 f   kernel32:KERNEL32.dll
 0002:00008308       _VirtualQuery@12           10019308 f   kernel32:KERNEL32.dll
 0002:0000830e       _FreeLibrary@4             1001930e f   kernel32:KERNEL32.dll
 0003:00000000       ___xc_a                    1001c000     MSVCRTD:cinitexe.obj
 0003:00000104       ___xc_z                    1001c104     MSVCRTD:cinitexe.obj
 0003:00000208       ___xi_a                    1001c208     MSVCRTD:cinitexe.obj
 0003:00000410       ___xi_z                    1001c410     MSVCRTD:cinitexe.obj
 0003:0000053c       ??_C@_0P@GHFPNOJB@bad?5allocation?$AA@ 1001c53c     IexBaseExc.obj
 0003:00000550       ?collate@?$_Locbase@H@std@@2HB 1001c550     IexBaseExc.obj
 0003:00000554       ?ctype@?$_Locbase@H@std@@2HB 1001c554     IexBaseExc.obj
 0003:00000558       ?monetary@?$_Locbase@H@std@@2HB 1001c558     IexBaseExc.obj
 0003:0000055c       ?numeric@?$_Locbase@H@std@@2HB 1001c55c     IexBaseExc.obj
 0003:00000560       ?time@?$_Locbase@H@std@@2HB 1001c560     IexBaseExc.obj
 0003:00000564       ?messages@?$_Locbase@H@std@@2HB 1001c564     IexBaseExc.obj
 0003:00000568       ?all@?$_Locbase@H@std@@2HB 1001c568     IexBaseExc.obj
 0003:0000056c       ?none@?$_Locbase@H@std@@2HB 1001c56c     IexBaseExc.obj
 0003:00000570       ?skipws@?$_Iosb@H@std@@2W4_Fmtflags@12@B 1001c570     IexBaseExc.obj
 0003:00000574       ?unitbuf@?$_Iosb@H@std@@2W4_Fmtflags@12@B 1001c574     IexBaseExc.obj
 0003:00000578       ?uppercase@?$_Iosb@H@std@@2W4_Fmtflags@12@B 1001c578     IexBaseExc.obj
 0003:0000057c       ?showbase@?$_Iosb@H@std@@2W4_Fmtflags@12@B 1001c57c     IexBaseExc.obj
 0003:00000580       ?showpoint@?$_Iosb@H@std@@2W4_Fmtflags@12@B 1001c580     IexBaseExc.obj
 0003:00000584       ?showpos@?$_Iosb@H@std@@2W4_Fmtflags@12@B 1001c584     IexBaseExc.obj
 0003:00000588       ?left@?$_Iosb@H@std@@2W4_Fmtflags@12@B 1001c588     IexBaseExc.obj
 0003:0000058c       ?right@?$_Iosb@H@std@@2W4_Fmtflags@12@B 1001c58c     IexBaseExc.obj
 0003:00000590       ?internal@?$_Iosb@H@std@@2W4_Fmtflags@12@B 1001c590     IexBaseExc.obj
 0003:00000594       ?dec@?$_Iosb@H@std@@2W4_Fmtflags@12@B 1001c594     IexBaseExc.obj
 0003:00000598       ?oct@?$_Iosb@H@std@@2W4_Fmtflags@12@B 1001c598     IexBaseExc.obj
 0003:0000059c       ?hex@?$_Iosb@H@std@@2W4_Fmtflags@12@B 1001c59c     IexBaseExc.obj
 0003:000005a0       ?scientific@?$_Iosb@H@std@@2W4_Fmtflags@12@B 1001c5a0     IexBaseExc.obj
 0003:000005a4       ?fixed@?$_Iosb@H@std@@2W4_Fmtflags@12@B 1001c5a4     IexBaseExc.obj
 0003:000005a8       ?boolalpha@?$_Iosb@H@std@@2W4_Fmtflags@12@B 1001c5a8     IexBaseExc.obj
 0003:000005ac       ?_Stdio@?$_Iosb@H@std@@2W4_Fmtflags@12@B 1001c5ac     IexBaseExc.obj
 0003:000005b0       ?adjustfield@?$_Iosb@H@std@@2W4_Fmtflags@12@B 1001c5b0     IexBaseExc.obj
 0003:000005b4       ?basefield@?$_Iosb@H@std@@2W4_Fmtflags@12@B 1001c5b4     IexBaseExc.obj
 0003:000005b8       ?floatfield@?$_Iosb@H@std@@2W4_Fmtflags@12@B 1001c5b8     IexBaseExc.obj
 0003:000005bc       ?goodbit@?$_Iosb@H@std@@2W4_Iostate@12@B 1001c5bc     IexBaseExc.obj
 0003:000005c0       ?eofbit@?$_Iosb@H@std@@2W4_Iostate@12@B 1001c5c0     IexBaseExc.obj
 0003:000005c4       ?failbit@?$_Iosb@H@std@@2W4_Iostate@12@B 1001c5c4     IexBaseExc.obj
 0003:000005c8       ?badbit@?$_Iosb@H@std@@2W4_Iostate@12@B 1001c5c8     IexBaseExc.obj
 0003:000005cc       ?_Hardfail@?$_Iosb@H@std@@2W4_Iostate@12@B 1001c5cc     IexBaseExc.obj
 0003:000005d0       ?in@?$_Iosb@H@std@@2W4_Openmode@12@B 1001c5d0     IexBaseExc.obj
 0003:000005d4       ?out@?$_Iosb@H@std@@2W4_Openmode@12@B 1001c5d4     IexBaseExc.obj
 0003:000005d8       ?ate@?$_Iosb@H@std@@2W4_Openmode@12@B 1001c5d8     IexBaseExc.obj
 0003:000005dc       ?app@?$_Iosb@H@std@@2W4_Openmode@12@B 1001c5dc     IexBaseExc.obj
 0003:000005e0       ?trunc@?$_Iosb@H@std@@2W4_Openmode@12@B 1001c5e0     IexBaseExc.obj
 0003:000005e4       ?_Nocreate@?$_Iosb@H@std@@2W4_Openmode@12@B 1001c5e4     IexBaseExc.obj
 0003:000005e8       ?_Noreplace@?$_Iosb@H@std@@2W4_Openmode@12@B 1001c5e8     IexBaseExc.obj
 0003:000005ec       ?binary@?$_Iosb@H@std@@2W4_Openmode@12@B 1001c5ec     IexBaseExc.obj
 0003:000005f0       ?beg@?$_Iosb@H@std@@2W4_Seekdir@12@B 1001c5f0     IexBaseExc.obj
 0003:000005f4       ?cur@?$_Iosb@H@std@@2W4_Seekdir@12@B 1001c5f4     IexBaseExc.obj
 0003:000005f8       ?end@?$_Iosb@H@std@@2W4_Seekdir@12@B 1001c5f8     IexBaseExc.obj
 0003:00000600       ??_7BaseExc@Iex@@6B@       1001c600     IexBaseExc.obj
 0003:0000060a       ??_C@_00CNPNBAHC@?$AA@     1001c60a     IexBaseExc.obj
 0003:0000060c       ??_C@_02OAOPDKLG@?$CFT?$AA@ 1001c60c     IexThrowErrnoExc.obj
 0003:00000614       ??_7ErrnoExc@Iex@@6B@      1001c614     IexThrowErrnoExc.obj
 0003:00000624       ??_7EpermExc@Iex@@6B@      1001c624     IexThrowErrnoExc.obj
 0003:00000634       ??_7EnoentExc@Iex@@6B@     1001c634     IexThrowErrnoExc.obj
 0003:00000644       ??_7EsrchExc@Iex@@6B@      1001c644     IexThrowErrnoExc.obj
 0003:00000654       ??_7EintrExc@Iex@@6B@      1001c654     IexThrowErrnoExc.obj
 0003:00000664       ??_7EioExc@Iex@@6B@        1001c664     IexThrowErrnoExc.obj
 0003:00000674       ??_7EnxioExc@Iex@@6B@      1001c674     IexThrowErrnoExc.obj
 0003:00000684       ??_7E2bigExc@Iex@@6B@      1001c684     IexThrowErrnoExc.obj
 0003:00000694       ??_7EnoexecExc@Iex@@6B@    1001c694     IexThrowErrnoExc.obj
 0003:000006a4       ??_7EbadfExc@Iex@@6B@      1001c6a4     IexThrowErrnoExc.obj
 0003:000006b4       ??_7EchildExc@Iex@@6B@     1001c6b4     IexThrowErrnoExc.obj
 0003:000006c4       ??_7EagainExc@Iex@@6B@     1001c6c4     IexThrowErrnoExc.obj
 0003:000006d4       ??_7EnomemExc@Iex@@6B@     1001c6d4     IexThrowErrnoExc.obj
 0003:000006e4       ??_7EaccesExc@Iex@@6B@     1001c6e4     IexThrowErrnoExc.obj
 0003:000006f4       ??_7EfaultExc@Iex@@6B@     1001c6f4     IexThrowErrnoExc.obj
 0003:00000704       ??_7EbusyExc@Iex@@6B@      1001c704     IexThrowErrnoExc.obj
 0003:00000714       ??_7EexistExc@Iex@@6B@     1001c714     IexThrowErrnoExc.obj
 0003:00000724       ??_7ExdevExc@Iex@@6B@      1001c724     IexThrowErrnoExc.obj
 0003:00000734       ??_7EnodevExc@Iex@@6B@     1001c734     IexThrowErrnoExc.obj
 0003:00000744       ??_7EnotdirExc@Iex@@6B@    1001c744     IexThrowErrnoExc.obj
 0003:00000754       ??_7EisdirExc@Iex@@6B@     1001c754     IexThrowErrnoExc.obj
 0003:00000764       ??_7EinvalExc@Iex@@6B@     1001c764     IexThrowErrnoExc.obj
 0003:00000774       ??_7EnfileExc@Iex@@6B@     1001c774     IexThrowErrnoExc.obj
 0003:00000784       ??_7EmfileExc@Iex@@6B@     1001c784     IexThrowErrnoExc.obj
 0003:00000794       ??_7EnottyExc@Iex@@6B@     1001c794     IexThrowErrnoExc.obj
 0003:000007a4       ??_7EfbigExc@Iex@@6B@      1001c7a4     IexThrowErrnoExc.obj
 0003:000007b4       ??_7EnospcExc@Iex@@6B@     1001c7b4     IexThrowErrnoExc.obj
 0003:000007c4       ??_7EspipeExc@Iex@@6B@     1001c7c4     IexThrowErrnoExc.obj
 0003:000007d4       ??_7ErofsExc@Iex@@6B@      1001c7d4     IexThrowErrnoExc.obj
 0003:000007e4       ??_7EmlinkExc@Iex@@6B@     1001c7e4     IexThrowErrnoExc.obj
 0003:000007f4       ??_7EpipeExc@Iex@@6B@      1001c7f4     IexThrowErrnoExc.obj
 0003:00000804       ??_7EdomExc@Iex@@6B@       1001c804     IexThrowErrnoExc.obj
 0003:00000814       ??_7ErangeExc@Iex@@6B@     1001c814     IexThrowErrnoExc.obj
 0003:00000824       ??_7EdeadlkExc@Iex@@6B@    1001c824     IexThrowErrnoExc.obj
 0003:00000834       ??_7EnolckExc@Iex@@6B@     1001c834     IexThrowErrnoExc.obj
 0003:00000844       ??_7EnametoolongExc@Iex@@6B@ 1001c844     IexThrowErrnoExc.obj
 0003:00000854       ??_7EilseqExc@Iex@@6B@     1001c854     IexThrowErrnoExc.obj
 0003:00000864       ??_7EnosysExc@Iex@@6B@     1001c864     IexThrowErrnoExc.obj
 0003:00000874       ??_7EnotemptyExc@Iex@@6B@  1001c874     IexThrowErrnoExc.obj
 0003:00000884       ??_7type_info@@6B@         1001c884     MSVCRTD:ti_inst.obj
 0003:0000088c       __pDefaultRawDllMain       1001c88c     MSVCRTD:crtdll.obj
 0003:0000088c       __pRawDllMain              1001c88c     MSVCRTD:crtdll.obj
 0003:00000890       ??_C@_08EIBOPINA@crtdll?4c?$AA@ 1001c890     MSVCRTD:crtdll.obj
 0003:0000089c       ??_C@_0BP@OGBCLIBO@Stack?5around?5_alloca?5corrupted?$AA@ 1001c89c     MSVCRTD:userapi.obj
 0003:000008c4       ??_C@_0CK@CNLNOEPB@Local?5variable?5used?5before?5initi@ 1001c8c4     MSVCRTD:userapi.obj
 0003:000008f8       ??_C@_0BI@CIGMDCBH@Stack?5memory?5corruption?$AA@ 1001c8f8     MSVCRTD:userapi.obj
 0003:00000914       ??_C@_0CK@FEGOIOPB@Cast?5to?5smaller?5type?5causing?5los@ 1001c914     MSVCRTD:userapi.obj
 0003:00000948       ??_C@_0BJ@HEGAHDFO@Stack?5pointer?5corruption?$AA@ 1001c948     MSVCRTD:userapi.obj
 0003:00000968       ??_C@_0BO@GNIAFIKK@Unknown?5Runtime?5Check?5Error?6?$AN?$AA@ 1001c968     MSVCRTD:error.obj
 0003:0000098c       ??_C@_0CM@NGINOKPC@Stack?5memory?5around?5_alloca?5was?5@ 1001c98c     MSVCRTD:error.obj
 0003:000009c0       ??_C@_0DG@HKJMLLLP@A?5local?5variable?5was?5used?5before@ 1001c9c0     MSVCRTD:error.obj
 0003:00000a00       ??_C@_0BN@FFOINMNJ@Stack?5memory?5was?5corrupted?6?$AN?$AA@ 1001ca00     MSVCRTD:error.obj
 0003:00000a28       ??_C@_0BBN@GPMLNJCF@A?5cast?5to?5a?5smaller?5data?5type?5ha@ 1001ca28     MSVCRTD:error.obj
 0003:00000b80       ??_C@_0NN@NGPKDKPD@The?5value?5of?5ESP?5was?5not?5properl@ 1001cb80     MSVCRTD:error.obj
 0003:00000d24       ??_C@_0CA@IODNCDPG@Run?9Time?5Check?5Failure?5?$CD?$CFd?5?9?5?$CFs?$AA@ 1001cd24     MSVCRTD:error.obj
 0003:00000d4c       ??_C@_0BE@GNBOBNCK@Unknown?5Module?5Name?$AA@ 1001cd4c     MSVCRTD:error.obj
 0003:00000d64       ??_C@_0BB@PFFGGCJP@Unknown?5Filename?$AA@ 1001cd64     MSVCRTD:error.obj
 0003:00000d78       ??_C@_1EA@NFKNIFJP@?$AAR?$AAu?$AAn?$AA?9?$AAT?$AAi?$AAm?$AAe?$AA?5?$AAC?$AAh?$AAe?$AAc?$AAk?$AA?5?$AAF?$AAa?$AAi?$AAl?$AAu?$AAr?$AAe?$AA?5?$AA?$CD?$AA?$CF?$AAd?$AA?5?$AA?9?$AA?5?$AA?$CF?$AAs?$AA?$AA@ 1001cd78     MSVCRTD:error.obj
 0003:00000dc8       ??_C@_1GM@OLMCBDMB@?$AAR?$AAu?$AAn?$AAt?$AAi?$AAm?$AAe?$AA?5?$AAC?$AAh?$AAe?$AAc?$AAk?$AA?5?$AAE?$AAr?$AAr?$AAo?$AAr?$AA?4?$AA?6?$AA?$AN?$AA?5?$AAU?$AAn?$AAa?$AAb?$AAl?$AAe?$AA?5?$AAt?$AAo@ 1001cdc8     MSVCRTD:error.obj
 0003:00000e4c       ??_C@_0CG@IAFNJNEE@Stack?5corrupted?5near?5unknown?5var@ 1001ce4c     MSVCRTD:error.obj
 0003:00000e80       ??_C@_0EJ@LJKNEOLN@Stack?5area?5around?5_alloca?5memory@ 1001ce80     MSVCRTD:error.obj
 0003:00000ed8       ??_C@_08KJEDNCKC@?$CFs?$CFs?$CFs?$CFs?$AA@ 1001ced8     MSVCRTD:error.obj
 0003:00000ee4       ??_C@_02LLMPMKNF@?$DO?5?$AA@ 1001cee4     MSVCRTD:error.obj
 0003:00000ee8       ??_C@_01EEMJAFIK@?6?$AA@   1001cee8     MSVCRTD:error.obj
 0003:00000eec       ??_C@_0BC@KIBAILCI@?$CFs?$CFs?$CFp?$CFs?$CFld?$CFs?$CFd?$CFs?$AA@ 1001ceec     MSVCRTD:error.obj
 0003:00000f08       ??_C@_0EI@CLEPFNGI@Stack?5area?5around?5_alloca?5memory@ 1001cf08     MSVCRTD:error.obj
 0003:00000f60       ??_C@_0N@MHFFIMFG@?6Address?3?50x?$AA@ 1001cf60     MSVCRTD:error.obj
 0003:00000f70       ??_C@_07DFDJCKFN@?6Size?3?5?$AA@ 1001cf70     MSVCRTD:error.obj
 0003:00000f7c       ??_C@_0CK@DKGBICFE@?6Allocation?5number?5within?5this?5f@ 1001cf7c     MSVCRTD:error.obj
 0003:00000fb0       ??_C@_08OMAHNMHJ@?6Data?3?5?$DM?$AA@ 1001cfb0     MSVCRTD:error.obj
 0003:00000fbc       ??_C@_09FOPFMPEJ@wsprintfA?$AA@ 1001cfbc     MSVCRTD:error.obj
 0003:00000fc8       ??_C@_0L@GMPLCCII@user32?4dll?$AA@ 1001cfc8     MSVCRTD:error.obj
 0003:00000fd8       ??_C@_05MKKEDADM@?$CF?42X?5?$AA@ 1001cfd8     MSVCRTD:error.obj
 0003:00000fe0       ??_C@_0DA@BEGFPCGG@A?5variable?5is?5being?5used?5without@ 1001cfe0     MSVCRTD:error.obj
 0003:00001028       ?ProcessDetach@NativeDll@<CrtImplementationDetails>@@0IB 1001d028     MSVCRTD:tncleanup.obj
 0003:0000102c       ?ProcessAttach@NativeDll@<CrtImplementationDetails>@@0IB 1001d02c     MSVCRTD:tncleanup.obj
 0003:00001030       ?ThreadAttach@NativeDll@<CrtImplementationDetails>@@0IB 1001d030     MSVCRTD:tncleanup.obj
 0003:00001034       ?ThreadDetach@NativeDll@<CrtImplementationDetails>@@0IB 1001d034     MSVCRTD:tncleanup.obj
 0003:00001038       ?ProcessVerifier@NativeDll@<CrtImplementationDetails>@@0IB 1001d038     MSVCRTD:tncleanup.obj
 0003:00001040       ??_C@_0OH@IHEJDJAH@Microsoft?5Visual?5C?$CL?$CL?5Runtime?5Lib@ 1001d040     MSVCRTD:gs_support.obj
 0003:00001158       ??_C@_0M@EKFFODEC@MSPDB80?4DLL?$AA@ 1001d158     MSVCRTD:pdblkup.obj
 0003:00001168       ??_C@_01KDCPPGHE@r?$AA@    1001d168     MSVCRTD:pdblkup.obj
 0003:0000116c       ??_C@_0BB@KCIACLNC@PDBOpenValidate5?$AA@ 1001d16c     MSVCRTD:pdblkup.obj
 0003:00001180       ??_C@_0BF@BMIHBHCA@EnvironmentDirectory?$AA@ 1001d180     MSVCRTD:pdblkup.obj
 0003:0000119c       ??_C@_0CN@EAEOKKOC@SOFTWARE?2Microsoft?2VisualStudio?2@ 1001d19c     MSVCRTD:pdblkup.obj
 0003:000011d4       ??_C@_0M@HLOHPNFA@RegCloseKey?$AA@ 1001d1d4     MSVCRTD:pdblkup.obj
 0003:000011e4       ??_C@_0BB@HHEIPGME@RegQueryValueExA?$AA@ 1001d1e4     MSVCRTD:pdblkup.obj
 0003:000011f8       ??_C@_0O@DCOGKJGG@RegOpenKeyExA?$AA@ 1001d1f8     MSVCRTD:pdblkup.obj
 0003:00001208       ??_C@_0N@JJPEKNFO@ADVAPI32?4DLL?$AA@ 1001d208     MSVCRTD:pdblkup.obj
 0003:000014e0       ??_R4BaseExc@Iex@@6B@      1001d4e0     IexBaseExc.obj
 0003:000014f8       ??_R3BaseExc@Iex@@8        1001d4f8     IexBaseExc.obj
 0003:0000150c       ??_R2BaseExc@Iex@@8        1001d50c     IexBaseExc.obj
 0003:0000152c       ??_R1A@?0A@EA@BaseExc@Iex@@8 1001d52c     IexBaseExc.obj
 0003:00001550       ??_R1M@?0A@EA@?$basic_string@DU?$char_traits@D@std@@V?$allocator@D@2@@std@@8 1001d550     IexBaseExc.obj
 0003:00001574       ??_R3?$basic_string@DU?$char_traits@D@std@@V?$allocator@D@2@@std@@8 1001d574     IexBaseExc.obj
 0003:00001588       ??_R2?$basic_string@DU?$char_traits@D@std@@V?$allocator@D@2@@std@@8 1001d588     IexBaseExc.obj
 0003:0000159c       ??_R1A@?0A@EA@?$basic_string@DU?$char_traits@D@std@@V?$allocator@D@2@@std@@8 1001d59c     IexBaseExc.obj
 0003:000015c0       ??_R1A@?0A@EA@?$_String_val@DV?$allocator@D@std@@@std@@8 1001d5c0     IexBaseExc.obj
 0003:000015e4       ??_R3?$_String_val@DV?$allocator@D@std@@@std@@8 1001d5e4     IexBaseExc.obj
 0003:000015f8       ??_R2?$_String_val@DV?$allocator@D@std@@@std@@8 1001d5f8     IexBaseExc.obj
 0003:00001608       ??_R1A@?0A@EA@_String_base@std@@8 1001d608     IexBaseExc.obj
 0003:0000162c       ??_R3_String_base@std@@8   1001d62c     IexBaseExc.obj
 0003:00001640       ??_R2_String_base@std@@8   1001d640     IexBaseExc.obj
 0003:0000164c       ??_R1A@?0A@EA@_Container_base@std@@8 1001d64c     IexBaseExc.obj
 0003:00001670       ??_R3_Container_base@std@@8 1001d670     IexBaseExc.obj
 0003:00001684       ??_R2_Container_base@std@@8 1001d684     IexBaseExc.obj
 0003:0000168c       ??_R1M@?0A@EA@?$_String_val@DV?$allocator@D@std@@@std@@8 1001d68c     IexBaseExc.obj
 0003:000016b0       ??_R1M@?0A@EA@_String_base@std@@8 1001d6b0     IexBaseExc.obj
 0003:000016d4       ??_R1M@?0A@EA@_Container_base@std@@8 1001d6d4     IexBaseExc.obj
 0003:000016f8       ??_R1A@?0A@EA@exception@std@@8 1001d6f8     IexBaseExc.obj
 0003:0000171c       ??_R3exception@std@@8      1001d71c     IexBaseExc.obj
 0003:00001730       ??_R2exception@std@@8      1001d730     IexBaseExc.obj
 0003:00001738       ??_R4ErrnoExc@Iex@@6B@     1001d738     IexThrowErrnoExc.obj
 0003:00001750       ??_R3ErrnoExc@Iex@@8       1001d750     IexThrowErrnoExc.obj
 0003:00001764       ??_R2ErrnoExc@Iex@@8       1001d764     IexThrowErrnoExc.obj
 0003:00001788       ??_R1A@?0A@EA@ErrnoExc@Iex@@8 1001d788     IexThrowErrnoExc.obj
 0003:000017ac       ??_R4EpermExc@Iex@@6B@     1001d7ac     IexThrowErrnoExc.obj
 0003:000017c4       ??_R3EpermExc@Iex@@8       1001d7c4     IexThrowErrnoExc.obj
 0003:000017d8       ??_R2EpermExc@Iex@@8       1001d7d8     IexThrowErrnoExc.obj
 0003:00001800       ??_R1A@?0A@EA@EpermExc@Iex@@8 1001d800     IexThrowErrnoExc.obj
 0003:00001824       ??_R4EnoentExc@Iex@@6B@    1001d824     IexThrowErrnoExc.obj
 0003:0000183c       ??_R3EnoentExc@Iex@@8      1001d83c     IexThrowErrnoExc.obj
 0003:00001850       ??_R2EnoentExc@Iex@@8      1001d850     IexThrowErrnoExc.obj
 0003:00001878       ??_R1A@?0A@EA@EnoentExc@Iex@@8 1001d878     IexThrowErrnoExc.obj
 0003:0000189c       ??_R4EsrchExc@Iex@@6B@     1001d89c     IexThrowErrnoExc.obj
 0003:000018b4       ??_R3EsrchExc@Iex@@8       1001d8b4     IexThrowErrnoExc.obj
 0003:000018c8       ??_R2EsrchExc@Iex@@8       1001d8c8     IexThrowErrnoExc.obj
 0003:000018f0       ??_R1A@?0A@EA@EsrchExc@Iex@@8 1001d8f0     IexThrowErrnoExc.obj
 0003:00001914       ??_R4EintrExc@Iex@@6B@     1001d914     IexThrowErrnoExc.obj
 0003:0000192c       ??_R3EintrExc@Iex@@8       1001d92c     IexThrowErrnoExc.obj
 0003:00001940       ??_R2EintrExc@Iex@@8       1001d940     IexThrowErrnoExc.obj
 0003:00001968       ??_R1A@?0A@EA@EintrExc@Iex@@8 1001d968     IexThrowErrnoExc.obj
 0003:0000198c       ??_R4EioExc@Iex@@6B@       1001d98c     IexThrowErrnoExc.obj
 0003:000019a4       ??_R3EioExc@Iex@@8         1001d9a4     IexThrowErrnoExc.obj
 0003:000019b8       ??_R2EioExc@Iex@@8         1001d9b8     IexThrowErrnoExc.obj
 0003:000019e0       ??_R1A@?0A@EA@EioExc@Iex@@8 1001d9e0     IexThrowErrnoExc.obj
 0003:00001a04       ??_R4EnxioExc@Iex@@6B@     1001da04     IexThrowErrnoExc.obj
 0003:00001a1c       ??_R3EnxioExc@Iex@@8       1001da1c     IexThrowErrnoExc.obj
 0003:00001a30       ??_R2EnxioExc@Iex@@8       1001da30     IexThrowErrnoExc.obj
 0003:00001a58       ??_R1A@?0A@EA@EnxioExc@Iex@@8 1001da58     IexThrowErrnoExc.obj
 0003:00001a7c       ??_R4E2bigExc@Iex@@6B@     1001da7c     IexThrowErrnoExc.obj
 0003:00001a94       ??_R3E2bigExc@Iex@@8       1001da94     IexThrowErrnoExc.obj
 0003:00001aa8       ??_R2E2bigExc@Iex@@8       1001daa8     IexThrowErrnoExc.obj
 0003:00001ad0       ??_R1A@?0A@EA@E2bigExc@Iex@@8 1001dad0     IexThrowErrnoExc.obj
 0003:00001af4       ??_R4EnoexecExc@Iex@@6B@   1001daf4     IexThrowErrnoExc.obj
 0003:00001b0c       ??_R3EnoexecExc@Iex@@8     1001db0c     IexThrowErrnoExc.obj
 0003:00001b20       ??_R2EnoexecExc@Iex@@8     1001db20     IexThrowErrnoExc.obj
 0003:00001b48       ??_R1A@?0A@EA@EnoexecExc@Iex@@8 1001db48     IexThrowErrnoExc.obj
 0003:00001b6c       ??_R4EbadfExc@Iex@@6B@     1001db6c     IexThrowErrnoExc.obj
 0003:00001b84       ??_R3EbadfExc@Iex@@8       1001db84     IexThrowErrnoExc.obj
 0003:00001b98       ??_R2EbadfExc@Iex@@8       1001db98     IexThrowErrnoExc.obj
 0003:00001bc0       ??_R1A@?0A@EA@EbadfExc@Iex@@8 1001dbc0     IexThrowErrnoExc.obj
 0003:00001be4       ??_R4EchildExc@Iex@@6B@    1001dbe4     IexThrowErrnoExc.obj
 0003:00001bfc       ??_R3EchildExc@Iex@@8      1001dbfc     IexThrowErrnoExc.obj
 0003:00001c10       ??_R2EchildExc@Iex@@8      1001dc10     IexThrowErrnoExc.obj
 0003:00001c38       ??_R1A@?0A@EA@EchildExc@Iex@@8 1001dc38     IexThrowErrnoExc.obj
 0003:00001c5c       ??_R4EagainExc@Iex@@6B@    1001dc5c     IexThrowErrnoExc.obj
 0003:00001c74       ??_R3EagainExc@Iex@@8      1001dc74     IexThrowErrnoExc.obj
 0003:00001c88       ??_R2EagainExc@Iex@@8      1001dc88     IexThrowErrnoExc.obj
 0003:00001cb0       ??_R1A@?0A@EA@EagainExc@Iex@@8 1001dcb0     IexThrowErrnoExc.obj
 0003:00001cd4       ??_R4EnomemExc@Iex@@6B@    1001dcd4     IexThrowErrnoExc.obj
 0003:00001cec       ??_R3EnomemExc@Iex@@8      1001dcec     IexThrowErrnoExc.obj
 0003:00001d00       ??_R2EnomemExc@Iex@@8      1001dd00     IexThrowErrnoExc.obj
 0003:00001d28       ??_R1A@?0A@EA@EnomemExc@Iex@@8 1001dd28     IexThrowErrnoExc.obj
 0003:00001d4c       ??_R4EaccesExc@Iex@@6B@    1001dd4c     IexThrowErrnoExc.obj
 0003:00001d64       ??_R3EaccesExc@Iex@@8      1001dd64     IexThrowErrnoExc.obj
 0003:00001d78       ??_R2EaccesExc@Iex@@8      1001dd78     IexThrowErrnoExc.obj
 0003:00001da0       ??_R1A@?0A@EA@EaccesExc@Iex@@8 1001dda0     IexThrowErrnoExc.obj
 0003:00001dc4       ??_R4EfaultExc@Iex@@6B@    1001ddc4     IexThrowErrnoExc.obj
 0003:00001ddc       ??_R3EfaultExc@Iex@@8      1001dddc     IexThrowErrnoExc.obj
 0003:00001df0       ??_R2EfaultExc@Iex@@8      1001ddf0     IexThrowErrnoExc.obj
 0003:00001e18       ??_R1A@?0A@EA@EfaultExc@Iex@@8 1001de18     IexThrowErrnoExc.obj
 0003:00001e3c       ??_R4EbusyExc@Iex@@6B@     1001de3c     IexThrowErrnoExc.obj
 0003:00001e54       ??_R3EbusyExc@Iex@@8       1001de54     IexThrowErrnoExc.obj
 0003:00001e68       ??_R2EbusyExc@Iex@@8       1001de68     IexThrowErrnoExc.obj
 0003:00001e90       ??_R1A@?0A@EA@EbusyExc@Iex@@8 1001de90     IexThrowErrnoExc.obj
 0003:00001eb4       ??_R4EexistExc@Iex@@6B@    1001deb4     IexThrowErrnoExc.obj
 0003:00001ecc       ??_R3EexistExc@Iex@@8      1001decc     IexThrowErrnoExc.obj
 0003:00001ee0       ??_R2EexistExc@Iex@@8      1001dee0     IexThrowErrnoExc.obj
 0003:00001f08       ??_R1A@?0A@EA@EexistExc@Iex@@8 1001df08     IexThrowErrnoExc.obj
 0003:00001f2c       ??_R4ExdevExc@Iex@@6B@     1001df2c     IexThrowErrnoExc.obj
 0003:00001f44       ??_R3ExdevExc@Iex@@8       1001df44     IexThrowErrnoExc.obj
 0003:00001f58       ??_R2ExdevExc@Iex@@8       1001df58     IexThrowErrnoExc.obj
 0003:00001f80       ??_R1A@?0A@EA@ExdevExc@Iex@@8 1001df80     IexThrowErrnoExc.obj
 0003:00001fa4       ??_R4EnodevExc@Iex@@6B@    1001dfa4     IexThrowErrnoExc.obj
 0003:00001fbc       ??_R3EnodevExc@Iex@@8      1001dfbc     IexThrowErrnoExc.obj
 0003:00001fd0       ??_R2EnodevExc@Iex@@8      1001dfd0     IexThrowErrnoExc.obj
 0003:00001ff8       ??_R1A@?0A@EA@EnodevExc@Iex@@8 1001dff8     IexThrowErrnoExc.obj
 0003:0000201c       ??_R4EnotdirExc@Iex@@6B@   1001e01c     IexThrowErrnoExc.obj
 0003:00002034       ??_R3EnotdirExc@Iex@@8     1001e034     IexThrowErrnoExc.obj
 0003:00002048       ??_R2EnotdirExc@Iex@@8     1001e048     IexThrowErrnoExc.obj
 0003:00002070       ??_R1A@?0A@EA@EnotdirExc@Iex@@8 1001e070     IexThrowErrnoExc.obj
 0003:00002094       ??_R4EisdirExc@Iex@@6B@    1001e094     IexThrowErrnoExc.obj
 0003:000020ac       ??_R3EisdirExc@Iex@@8      1001e0ac     IexThrowErrnoExc.obj
 0003:000020c0       ??_R2EisdirExc@Iex@@8      1001e0c0     IexThrowErrnoExc.obj
 0003:000020e8       ??_R1A@?0A@EA@EisdirExc@Iex@@8 1001e0e8     IexThrowErrnoExc.obj
 0003:0000210c       ??_R4EinvalExc@Iex@@6B@    1001e10c     IexThrowErrnoExc.obj
 0003:00002124       ??_R3EinvalExc@Iex@@8      1001e124     IexThrowErrnoExc.obj
 0003:00002138       ??_R2EinvalExc@Iex@@8      1001e138     IexThrowErrnoExc.obj
 0003:00002160       ??_R1A@?0A@EA@EinvalExc@Iex@@8 1001e160     IexThrowErrnoExc.obj
 0003:00002184       ??_R4EnfileExc@Iex@@6B@    1001e184     IexThrowErrnoExc.obj
 0003:0000219c       ??_R3EnfileExc@Iex@@8      1001e19c     IexThrowErrnoExc.obj
 0003:000021b0       ??_R2EnfileExc@Iex@@8      1001e1b0     IexThrowErrnoExc.obj
 0003:000021d8       ??_R1A@?0A@EA@EnfileExc@Iex@@8 1001e1d8     IexThrowErrnoExc.obj
 0003:000021fc       ??_R4EmfileExc@Iex@@6B@    1001e1fc     IexThrowErrnoExc.obj
 0003:00002214       ??_R3EmfileExc@Iex@@8      1001e214     IexThrowErrnoExc.obj
 0003:00002228       ??_R2EmfileExc@Iex@@8      1001e228     IexThrowErrnoExc.obj
 0003:00002250       ??_R1A@?0A@EA@EmfileExc@Iex@@8 1001e250     IexThrowErrnoExc.obj
 0003:00002274       ??_R4EnottyExc@Iex@@6B@    1001e274     IexThrowErrnoExc.obj
 0003:0000228c       ??_R3EnottyExc@Iex@@8      1001e28c     IexThrowErrnoExc.obj
 0003:000022a0       ??_R2EnottyExc@Iex@@8      1001e2a0     IexThrowErrnoExc.obj
 0003:000022c8       ??_R1A@?0A@EA@EnottyExc@Iex@@8 1001e2c8     IexThrowErrnoExc.obj
 0003:000022ec       ??_R4EfbigExc@Iex@@6B@     1001e2ec     IexThrowErrnoExc.obj
 0003:00002304       ??_R3EfbigExc@Iex@@8       1001e304     IexThrowErrnoExc.obj
 0003:00002318       ??_R2EfbigExc@Iex@@8       1001e318     IexThrowErrnoExc.obj
 0003:00002340       ??_R1A@?0A@EA@EfbigExc@Iex@@8 1001e340     IexThrowErrnoExc.obj
 0003:00002364       ??_R4EnospcExc@Iex@@6B@    1001e364     IexThrowErrnoExc.obj
 0003:0000237c       ??_R3EnospcExc@Iex@@8      1001e37c     IexThrowErrnoExc.obj
 0003:00002390       ??_R2EnospcExc@Iex@@8      1001e390     IexThrowErrnoExc.obj
 0003:000023b8       ??_R1A@?0A@EA@EnospcExc@Iex@@8 1001e3b8     IexThrowErrnoExc.obj
 0003:000023dc       ??_R4EspipeExc@Iex@@6B@    1001e3dc     IexThrowErrnoExc.obj
 0003:000023f4       ??_R3EspipeExc@Iex@@8      1001e3f4     IexThrowErrnoExc.obj
 0003:00002408       ??_R2EspipeExc@Iex@@8      1001e408     IexThrowErrnoExc.obj
 0003:00002430       ??_R1A@?0A@EA@EspipeExc@Iex@@8 1001e430     IexThrowErrnoExc.obj
 0003:00002454       ??_R4ErofsExc@Iex@@6B@     1001e454     IexThrowErrnoExc.obj
 0003:0000246c       ??_R3ErofsExc@Iex@@8       1001e46c     IexThrowErrnoExc.obj
 0003:00002480       ??_R2ErofsExc@Iex@@8       1001e480     IexThrowErrnoExc.obj
 0003:000024a8       ??_R1A@?0A@EA@ErofsExc@Iex@@8 1001e4a8     IexThrowErrnoExc.obj
 0003:000024cc       ??_R4EmlinkExc@Iex@@6B@    1001e4cc     IexThrowErrnoExc.obj
 0003:000024e4       ??_R3EmlinkExc@Iex@@8      1001e4e4     IexThrowErrnoExc.obj
 0003:000024f8       ??_R2EmlinkExc@Iex@@8      1001e4f8     IexThrowErrnoExc.obj
 0003:00002520       ??_R1A@?0A@EA@EmlinkExc@Iex@@8 1001e520     IexThrowErrnoExc.obj
 0003:00002544       ??_R4EpipeExc@Iex@@6B@     1001e544     IexThrowErrnoExc.obj
 0003:0000255c       ??_R3EpipeExc@Iex@@8       1001e55c     IexThrowErrnoExc.obj
 0003:00002570       ??_R2EpipeExc@Iex@@8       1001e570     IexThrowErrnoExc.obj
 0003:00002598       ??_R1A@?0A@EA@EpipeExc@Iex@@8 1001e598     IexThrowErrnoExc.obj
 0003:000025bc       ??_R4EdomExc@Iex@@6B@      1001e5bc     IexThrowErrnoExc.obj
 0003:000025d4       ??_R3EdomExc@Iex@@8        1001e5d4     IexThrowErrnoExc.obj
 0003:000025e8       ??_R2EdomExc@Iex@@8        1001e5e8     IexThrowErrnoExc.obj
 0003:00002610       ??_R1A@?0A@EA@EdomExc@Iex@@8 1001e610     IexThrowErrnoExc.obj
 0003:00002634       ??_R4ErangeExc@Iex@@6B@    1001e634     IexThrowErrnoExc.obj
 0003:0000264c       ??_R3ErangeExc@Iex@@8      1001e64c     IexThrowErrnoExc.obj
 0003:00002660       ??_R2ErangeExc@Iex@@8      1001e660     IexThrowErrnoExc.obj
 0003:00002688       ??_R1A@?0A@EA@ErangeExc@Iex@@8 1001e688     IexThrowErrnoExc.obj
 0003:000026ac       ??_R4EdeadlkExc@Iex@@6B@   1001e6ac     IexThrowErrnoExc.obj
 0003:000026c4       ??_R3EdeadlkExc@Iex@@8     1001e6c4     IexThrowErrnoExc.obj
 0003:000026d8       ??_R2EdeadlkExc@Iex@@8     1001e6d8     IexThrowErrnoExc.obj
 0003:00002700       ??_R1A@?0A@EA@EdeadlkExc@Iex@@8 1001e700     IexThrowErrnoExc.obj
 0003:00002724       ??_R4EnolckExc@Iex@@6B@    1001e724     IexThrowErrnoExc.obj
 0003:0000273c       ??_R3EnolckExc@Iex@@8      1001e73c     IexThrowErrnoExc.obj
 0003:00002750       ??_R2EnolckExc@Iex@@8      1001e750     IexThrowErrnoExc.obj
 0003:00002778       ??_R1A@?0A@EA@EnolckExc@Iex@@8 1001e778     IexThrowErrnoExc.obj
 0003:0000279c       ??_R4EnametoolongExc@Iex@@6B@ 1001e79c     IexThrowErrnoExc.obj
 0003:000027b4       ??_R3EnametoolongExc@Iex@@8 1001e7b4     IexThrowErrnoExc.obj
 0003:000027c8       ??_R2EnametoolongExc@Iex@@8 1001e7c8     IexThrowErrnoExc.obj
 0003:000027f0       ??_R1A@?0A@EA@EnametoolongExc@Iex@@8 1001e7f0     IexThrowErrnoExc.obj
 0003:00002814       ??_R4EilseqExc@Iex@@6B@    1001e814     IexThrowErrnoExc.obj
 0003:0000282c       ??_R3EilseqExc@Iex@@8      1001e82c     IexThrowErrnoExc.obj
 0003:00002840       ??_R2EilseqExc@Iex@@8      1001e840     IexThrowErrnoExc.obj
 0003:00002868       ??_R1A@?0A@EA@EilseqExc@Iex@@8 1001e868     IexThrowErrnoExc.obj
 0003:0000288c       ??_R4EnosysExc@Iex@@6B@    1001e88c     IexThrowErrnoExc.obj
 0003:000028a4       ??_R3EnosysExc@Iex@@8      1001e8a4     IexThrowErrnoExc.obj
 0003:000028b8       ??_R2EnosysExc@Iex@@8      1001e8b8     IexThrowErrnoExc.obj
 0003:000028e0       ??_R1A@?0A@EA@EnosysExc@Iex@@8 1001e8e0     IexThrowErrnoExc.obj
 0003:00002904       ??_R4EnotemptyExc@Iex@@6B@ 1001e904     IexThrowErrnoExc.obj
 0003:0000291c       ??_R3EnotemptyExc@Iex@@8   1001e91c     IexThrowErrnoExc.obj
 0003:00002930       ??_R2EnotemptyExc@Iex@@8   1001e930     IexThrowErrnoExc.obj
 0003:00002958       ??_R1A@?0A@EA@EnotemptyExc@Iex@@8 1001e958     IexThrowErrnoExc.obj
 0003:0000297c       ??_R4type_info@@6B@        1001e97c     MSVCRTD:ti_inst.obj
 0003:00002994       ??_R3type_info@@8          1001e994     MSVCRTD:ti_inst.obj
 0003:000029a8       ??_R2type_info@@8          1001e9a8     MSVCRTD:ti_inst.obj
 0003:000029b0       ??_R1A@?0A@EA@type_info@@8 1001e9b0     MSVCRTD:ti_inst.obj
 0003:00002b44       ___rtc_iaa                 1001eb44     MSVCRTD:initsect.obj
 0003:00002d54       ___rtc_izz                 1001ed54     MSVCRTD:initsect.obj
 0003:00002e58       ___rtc_taa                 1001ee58     MSVCRTD:initsect.obj
 0003:00003068       ___rtc_tzz                 1001f068     MSVCRTD:initsect.obj
 0003:000031d0       __TI7?AVErrnoExc@Iex@@     1001f1d0     IexThrowErrnoExc.obj
 0003:000031e4       __TI8?AVEnotemptyExc@Iex@@ 1001f1e4     IexThrowErrnoExc.obj
 0003:000031f8       __TI8?AVEnosysExc@Iex@@    1001f1f8     IexThrowErrnoExc.obj
 0003:0000320c       __TI8?AVEilseqExc@Iex@@    1001f20c     IexThrowErrnoExc.obj
 0003:00003220       __TI8?AVEnametoolongExc@Iex@@ 1001f220     IexThrowErrnoExc.obj
 0003:00003234       __TI8?AVEnolckExc@Iex@@    1001f234     IexThrowErrnoExc.obj
 0003:00003248       __TI8?AVEdeadlkExc@Iex@@   1001f248     IexThrowErrnoExc.obj
 0003:0000325c       __TI8?AVErangeExc@Iex@@    1001f25c     IexThrowErrnoExc.obj
 0003:00003270       __TI8?AVEdomExc@Iex@@      1001f270     IexThrowErrnoExc.obj
 0003:00003284       __TI8?AVEpipeExc@Iex@@     1001f284     IexThrowErrnoExc.obj
 0003:00003298       __TI8?AVEmlinkExc@Iex@@    1001f298     IexThrowErrnoExc.obj
 0003:000032ac       __TI8?AVErofsExc@Iex@@     1001f2ac     IexThrowErrnoExc.obj
 0003:000032c0       __TI8?AVEspipeExc@Iex@@    1001f2c0     IexThrowErrnoExc.obj
 0003:000032d4       __TI8?AVEnospcExc@Iex@@    1001f2d4     IexThrowErrnoExc.obj
 0003:000032e8       __TI8?AVEfbigExc@Iex@@     1001f2e8     IexThrowErrnoExc.obj
 0003:000032fc       __TI8?AVEnottyExc@Iex@@    1001f2fc     IexThrowErrnoExc.obj
 0003:00003310       __TI8?AVEmfileExc@Iex@@    1001f310     IexThrowErrnoExc.obj
 0003:00003324       __TI8?AVEnfileExc@Iex@@    1001f324     IexThrowErrnoExc.obj
 0003:00003338       __TI8?AVEinvalExc@Iex@@    1001f338     IexThrowErrnoExc.obj
 0003:0000334c       __TI8?AVEisdirExc@Iex@@    1001f34c     IexThrowErrnoExc.obj
 0003:00003360       __TI8?AVEnotdirExc@Iex@@   1001f360     IexThrowErrnoExc.obj
 0003:00003374       __TI8?AVEnodevExc@Iex@@    1001f374     IexThrowErrnoExc.obj
 0003:00003388       __TI8?AVExdevExc@Iex@@     1001f388     IexThrowErrnoExc.obj
 0003:0000339c       __TI8?AVEexistExc@Iex@@    1001f39c     IexThrowErrnoExc.obj
 0003:000033b0       __TI8?AVEbusyExc@Iex@@     1001f3b0     IexThrowErrnoExc.obj
 0003:000033c4       __TI8?AVEfaultExc@Iex@@    1001f3c4     IexThrowErrnoExc.obj
 0003:000033d8       __TI8?AVEaccesExc@Iex@@    1001f3d8     IexThrowErrnoExc.obj
 0003:000033ec       __TI8?AVEnomemExc@Iex@@    1001f3ec     IexThrowErrnoExc.obj
 0003:00003400       __TI8?AVEagainExc@Iex@@    1001f400     IexThrowErrnoExc.obj
 0003:00003414       __TI8?AVEchildExc@Iex@@    1001f414     IexThrowErrnoExc.obj
 0003:00003428       __TI8?AVEbadfExc@Iex@@     1001f428     IexThrowErrnoExc.obj
 0003:0000343c       __TI8?AVEnoexecExc@Iex@@   1001f43c     IexThrowErrnoExc.obj
 0003:00003450       __TI8?AVE2bigExc@Iex@@     1001f450     IexThrowErrnoExc.obj
 0003:00003464       __TI8?AVEnxioExc@Iex@@     1001f464     IexThrowErrnoExc.obj
 0003:00003478       __TI8?AVEioExc@Iex@@       1001f478     IexThrowErrnoExc.obj
 0003:0000348c       __TI8?AVEintrExc@Iex@@     1001f48c     IexThrowErrnoExc.obj
 0003:000034a0       __TI8?AVEsrchExc@Iex@@     1001f4a0     IexThrowErrnoExc.obj
 0003:000034b4       __TI8?AVEnoentExc@Iex@@    1001f4b4     IexThrowErrnoExc.obj
 0003:000034c8       __TI8?AVEpermExc@Iex@@     1001f4c8     IexThrowErrnoExc.obj
 0003:0000350c       __CTA8?AVEpermExc@Iex@@    1001f50c     IexThrowErrnoExc.obj
 0003:00003534       __CT??_R0?AVEpermExc@Iex@@@8??0EpermExc@Iex@@QAE@ABV01@@Z76 1001f534     IexThrowErrnoExc.obj
 0003:00003554       __CT??_R0?AVErrnoExc@Iex@@@8??0ErrnoExc@Iex@@QAE@ABV01@@Z76 1001f554     IexThrowErrnoExc.obj
 0003:00003574       __CT??_R0?AVBaseExc@Iex@@@8??0BaseExc@Iex@@QAE@ABV01@@Z76 1001f574     IexThrowErrnoExc.obj
 0003:00003594       __CT??_R0?AV?$basic_string@DU?$char_traits@D@std@@V?$allocator@D@2@@std@@@8??0?$basic_string@DU?$char_traits@D@std@@V?$allocator@D@2@@std@@QAE@ABV01@@Z3212 1001f594     IexThrowErrnoExc.obj
 0003:000035b4       __CT??_R0?AV?$_String_val@DV?$allocator@D@std@@@std@@@8??0?$_String_val@DV?$allocator@D@std@@@std@@QAE@ABV01@@Z812 1001f5b4     IexThrowErrnoExc.obj
 0003:000035d4       __CT??_R0?AV_String_base@std@@@8??0_String_base@std@@QAE@ABV01@@Z412 1001f5d4     IexThrowErrnoExc.obj
 0003:000035f4       __CT??_R0?AV_Container_base@std@@@8??0_Container_base@std@@QAE@ABV01@@Z412 1001f5f4     IexThrowErrnoExc.obj
 0003:00003614       __CT??_R0?AVexception@std@@@8??0exception@std@@QAE@ABV01@@Z12 1001f614     IexThrowErrnoExc.obj
 0003:00003634       __CTA8?AVEnoentExc@Iex@@   1001f634     IexThrowErrnoExc.obj
 0003:0000365c       __CT??_R0?AVEnoentExc@Iex@@@8??0EnoentExc@Iex@@QAE@ABV01@@Z76 1001f65c     IexThrowErrnoExc.obj
 0003:0000367c       __CTA8?AVEsrchExc@Iex@@    1001f67c     IexThrowErrnoExc.obj
 0003:000036a4       __CT??_R0?AVEsrchExc@Iex@@@8??0EsrchExc@Iex@@QAE@ABV01@@Z76 1001f6a4     IexThrowErrnoExc.obj
 0003:000036c4       __CTA8?AVEintrExc@Iex@@    1001f6c4     IexThrowErrnoExc.obj
 0003:000036ec       __CT??_R0?AVEintrExc@Iex@@@8??0EintrExc@Iex@@QAE@ABV01@@Z76 1001f6ec     IexThrowErrnoExc.obj
 0003:0000370c       __CTA8?AVEioExc@Iex@@      1001f70c     IexThrowErrnoExc.obj
 0003:00003734       __CT??_R0?AVEioExc@Iex@@@8??0EioExc@Iex@@QAE@ABV01@@Z76 1001f734     IexThrowErrnoExc.obj
 0003:00003754       __CTA8?AVEnxioExc@Iex@@    1001f754     IexThrowErrnoExc.obj
 0003:0000377c       __CT??_R0?AVEnxioExc@Iex@@@8??0EnxioExc@Iex@@QAE@ABV01@@Z76 1001f77c     IexThrowErrnoExc.obj
 0003:0000379c       __CTA8?AVE2bigExc@Iex@@    1001f79c     IexThrowErrnoExc.obj
 0003:000037c4       __CT??_R0?AVE2bigExc@Iex@@@8??0E2bigExc@Iex@@QAE@ABV01@@Z76 1001f7c4     IexThrowErrnoExc.obj
 0003:000037e4       __CTA8?AVEnoexecExc@Iex@@  1001f7e4     IexThrowErrnoExc.obj
 0003:0000380c       __CT??_R0?AVEnoexecExc@Iex@@@8??0EnoexecExc@Iex@@QAE@ABV01@@Z76 1001f80c     IexThrowErrnoExc.obj
 0003:0000382c       __CTA8?AVEbadfExc@Iex@@    1001f82c     IexThrowErrnoExc.obj
 0003:00003854       __CT??_R0?AVEbadfExc@Iex@@@8??0EbadfExc@Iex@@QAE@ABV01@@Z76 1001f854     IexThrowErrnoExc.obj
 0003:00003874       __CTA8?AVEchildExc@Iex@@   1001f874     IexThrowErrnoExc.obj
 0003:0000389c       __CT??_R0?AVEchildExc@Iex@@@8??0EchildExc@Iex@@QAE@ABV01@@Z76 1001f89c     IexThrowErrnoExc.obj
 0003:000038bc       __CTA8?AVEagainExc@Iex@@   1001f8bc     IexThrowErrnoExc.obj
 0003:000038e4       __CT??_R0?AVEagainExc@Iex@@@8??0EagainExc@Iex@@QAE@ABV01@@Z76 1001f8e4     IexThrowErrnoExc.obj
 0003:00003904       __CTA8?AVEnomemExc@Iex@@   1001f904     IexThrowErrnoExc.obj
 0003:0000392c       __CT??_R0?AVEnomemExc@Iex@@@8??0EnomemExc@Iex@@QAE@ABV01@@Z76 1001f92c     IexThrowErrnoExc.obj
 0003:0000394c       __CTA8?AVEaccesExc@Iex@@   1001f94c     IexThrowErrnoExc.obj
 0003:00003974       __CT??_R0?AVEaccesExc@Iex@@@8??0EaccesExc@Iex@@QAE@ABV01@@Z76 1001f974     IexThrowErrnoExc.obj
 0003:00003994       __CTA8?AVEfaultExc@Iex@@   1001f994     IexThrowErrnoExc.obj
 0003:000039bc       __CT??_R0?AVEfaultExc@Iex@@@8??0EfaultExc@Iex@@QAE@ABV01@@Z76 1001f9bc     IexThrowErrnoExc.obj
 0003:000039dc       __CTA8?AVEbusyExc@Iex@@    1001f9dc     IexThrowErrnoExc.obj
 0003:00003a04       __CT??_R0?AVEbusyExc@Iex@@@8??0EbusyExc@Iex@@QAE@ABV01@@Z76 1001fa04     IexThrowErrnoExc.obj
 0003:00003a24       __CTA8?AVEexistExc@Iex@@   1001fa24     IexThrowErrnoExc.obj
 0003:00003a4c       __CT??_R0?AVEexistExc@Iex@@@8??0EexistExc@Iex@@QAE@ABV01@@Z76 1001fa4c     IexThrowErrnoExc.obj
 0003:00003a6c       __CTA8?AVExdevExc@Iex@@    1001fa6c     IexThrowErrnoExc.obj
 0003:00003a94       __CT??_R0?AVExdevExc@Iex@@@8??0ExdevExc@Iex@@QAE@ABV01@@Z76 1001fa94     IexThrowErrnoExc.obj
 0003:00003ab4       __CTA8?AVEnodevExc@Iex@@   1001fab4     IexThrowErrnoExc.obj
 0003:00003adc       __CT??_R0?AVEnodevExc@Iex@@@8??0EnodevExc@Iex@@QAE@ABV01@@Z76 1001fadc     IexThrowErrnoExc.obj
 0003:00003afc       __CTA8?AVEnotdirExc@Iex@@  1001fafc     IexThrowErrnoExc.obj
 0003:00003b24       __CT??_R0?AVEnotdirExc@Iex@@@8??0EnotdirExc@Iex@@QAE@ABV01@@Z76 1001fb24     IexThrowErrnoExc.obj
 0003:00003b44       __CTA8?AVEisdirExc@Iex@@   1001fb44     IexThrowErrnoExc.obj
 0003:00003b6c       __CT??_R0?AVEisdirExc@Iex@@@8??0EisdirExc@Iex@@QAE@ABV01@@Z76 1001fb6c     IexThrowErrnoExc.obj
 0003:00003b8c       __CTA8?AVEinvalExc@Iex@@   1001fb8c     IexThrowErrnoExc.obj
 0003:00003bb4       __CT??_R0?AVEinvalExc@Iex@@@8??0EinvalExc@Iex@@QAE@ABV01@@Z76 1001fbb4     IexThrowErrnoExc.obj
 0003:00003bd4       __CTA8?AVEnfileExc@Iex@@   1001fbd4     IexThrowErrnoExc.obj
 0003:00003bfc       __CT??_R0?AVEnfileExc@Iex@@@8??0EnfileExc@Iex@@QAE@ABV01@@Z76 1001fbfc     IexThrowErrnoExc.obj
 0003:00003c1c       __CTA8?AVEmfileExc@Iex@@   1001fc1c     IexThrowErrnoExc.obj
 0003:00003c44       __CT??_R0?AVEmfileExc@Iex@@@8??0EmfileExc@Iex@@QAE@ABV01@@Z76 1001fc44     IexThrowErrnoExc.obj
 0003:00003c64       __CTA8?AVEnottyExc@Iex@@   1001fc64     IexThrowErrnoExc.obj
 0003:00003c8c       __CT??_R0?AVEnottyExc@Iex@@@8??0EnottyExc@Iex@@QAE@ABV01@@Z76 1001fc8c     IexThrowErrnoExc.obj
 0003:00003cac       __CTA8?AVEfbigExc@Iex@@    1001fcac     IexThrowErrnoExc.obj
 0003:00003cd4       __CT??_R0?AVEfbigExc@Iex@@@8??0EfbigExc@Iex@@QAE@ABV01@@Z76 1001fcd4     IexThrowErrnoExc.obj
 0003:00003cf4       __CTA8?AVEnospcExc@Iex@@   1001fcf4     IexThrowErrnoExc.obj
 0003:00003d1c       __CT??_R0?AVEnospcExc@Iex@@@8??0EnospcExc@Iex@@QAE@ABV01@@Z76 1001fd1c     IexThrowErrnoExc.obj
 0003:00003d3c       __CTA8?AVEspipeExc@Iex@@   1001fd3c     IexThrowErrnoExc.obj
 0003:00003d64       __CT??_R0?AVEspipeExc@Iex@@@8??0EspipeExc@Iex@@QAE@ABV01@@Z76 1001fd64     IexThrowErrnoExc.obj
 0003:00003d84       __CTA8?AVErofsExc@Iex@@    1001fd84     IexThrowErrnoExc.obj
 0003:00003dac       __CT??_R0?AVErofsExc@Iex@@@8??0ErofsExc@Iex@@QAE@ABV01@@Z76 1001fdac     IexThrowErrnoExc.obj
 0003:00003dcc       __CTA8?AVEmlinkExc@Iex@@   1001fdcc     IexThrowErrnoExc.obj
 0003:00003df4       __CT??_R0?AVEmlinkExc@Iex@@@8??0EmlinkExc@Iex@@QAE@ABV01@@Z76 1001fdf4     IexThrowErrnoExc.obj
 0003:00003e14       __CTA8?AVEpipeExc@Iex@@    1001fe14     IexThrowErrnoExc.obj
 0003:00003e3c       __CT??_R0?AVEpipeExc@Iex@@@8??0EpipeExc@Iex@@QAE@ABV01@@Z76 1001fe3c     IexThrowErrnoExc.obj
 0003:00003e5c       __CTA8?AVEdomExc@Iex@@     1001fe5c     IexThrowErrnoExc.obj
 0003:00003e84       __CT??_R0?AVEdomExc@Iex@@@8??0EdomExc@Iex@@QAE@ABV01@@Z76 1001fe84     IexThrowErrnoExc.obj
 0003:00003ea4       __CTA8?AVErangeExc@Iex@@   1001fea4     IexThrowErrnoExc.obj
 0003:00003ecc       __CT??_R0?AVErangeExc@Iex@@@8??0ErangeExc@Iex@@QAE@ABV01@@Z76 1001fecc     IexThrowErrnoExc.obj
 0003:00003eec       __CTA8?AVEdeadlkExc@Iex@@  1001feec     IexThrowErrnoExc.obj
 0003:00003f14       __CT??_R0?AVEdeadlkExc@Iex@@@8??0EdeadlkExc@Iex@@QAE@ABV01@@Z76 1001ff14     IexThrowErrnoExc.obj
 0003:00003f34       __CTA8?AVEnolckExc@Iex@@   1001ff34     IexThrowErrnoExc.obj
 0003:00003f5c       __CT??_R0?AVEnolckExc@Iex@@@8??0EnolckExc@Iex@@QAE@ABV01@@Z76 1001ff5c     IexThrowErrnoExc.obj
 0003:00003f7c       __CTA8?AVEnametoolongExc@Iex@@ 1001ff7c     IexThrowErrnoExc.obj
 0003:00003fa4       __CT??_R0?AVEnametoolongExc@Iex@@@8??0EnametoolongExc@Iex@@QAE@ABV01@@Z76 1001ffa4     IexThrowErrnoExc.obj
 0003:00003fc4       __CTA8?AVEilseqExc@Iex@@   1001ffc4     IexThrowErrnoExc.obj
 0003:00003fec       __CT??_R0?AVEilseqExc@Iex@@@8??0EilseqExc@Iex@@QAE@ABV01@@Z76 1001ffec     IexThrowErrnoExc.obj
 0003:0000400c       __CTA8?AVEnosysExc@Iex@@   1002000c     IexThrowErrnoExc.obj
 0003:00004034       __CT??_R0?AVEnosysExc@Iex@@@8??0EnosysExc@Iex@@QAE@ABV01@@Z76 10020034     IexThrowErrnoExc.obj
 0003:00004054       __CTA8?AVEnotemptyExc@Iex@@ 10020054     IexThrowErrnoExc.obj
 0003:0000407c       __CT??_R0?AVEnotemptyExc@Iex@@@8??0EnotemptyExc@Iex@@QAE@ABV01@@Z76 1002007c     IexThrowErrnoExc.obj
 0003:0000409c       __CTA7?AVErrnoExc@Iex@@    1002009c     IexThrowErrnoExc.obj
 0004:00000004       ??_R0?AVBaseExc@Iex@@@8    10021004     IexBaseExc.obj
 0004:00000028       ??_R0?AV?$basic_string@DU?$char_traits@D@std@@V?$allocator@D@2@@std@@@8 10021028     IexBaseExc.obj
 0004:00000080       ??_R0?AV?$_String_val@DV?$allocator@D@std@@@std@@@8 10021080     IexBaseExc.obj
 0004:000000c0       ??_R0?AV_String_base@std@@@8 100210c0     IexBaseExc.obj
 0004:000000e8       ??_R0?AV_Container_base@std@@@8 100210e8     IexBaseExc.obj
 0004:00000110       ??_R0?AVexception@std@@@8  10021110     IexBaseExc.obj
 0004:00000138       ??_R0?AVEpermExc@Iex@@@8   10021138     IexThrowErrnoExc.obj
 0004:00000158       ??_R0?AVErrnoExc@Iex@@@8   10021158     IexThrowErrnoExc.obj
 0004:00000178       ??_R0?AVEnoentExc@Iex@@@8  10021178     IexThrowErrnoExc.obj
 0004:0000019c       ??_R0?AVEsrchExc@Iex@@@8   1002119c     IexThrowErrnoExc.obj
 0004:000001bc       ??_R0?AVEintrExc@Iex@@@8   100211bc     IexThrowErrnoExc.obj
 0004:000001dc       ??_R0?AVEioExc@Iex@@@8     100211dc     IexThrowErrnoExc.obj
 0004:000001fc       ??_R0?AVEnxioExc@Iex@@@8   100211fc     IexThrowErrnoExc.obj
 0004:0000021c       ??_R0?AVE2bigExc@Iex@@@8   1002121c     IexThrowErrnoExc.obj
 0004:0000023c       ??_R0?AVEnoexecExc@Iex@@@8 1002123c     IexThrowErrnoExc.obj
 0004:00000260       ??_R0?AVEbadfExc@Iex@@@8   10021260     IexThrowErrnoExc.obj
 0004:00000280       ??_R0?AVEchildExc@Iex@@@8  10021280     IexThrowErrnoExc.obj
 0004:000002a4       ??_R0?AVEagainExc@Iex@@@8  100212a4     IexThrowErrnoExc.obj
 0004:000002c8       ??_R0?AVEnomemExc@Iex@@@8  100212c8     IexThrowErrnoExc.obj
 0004:000002ec       ??_R0?AVEaccesExc@Iex@@@8  100212ec     IexThrowErrnoExc.obj
 0004:00000310       ??_R0?AVEfaultExc@Iex@@@8  10021310     IexThrowErrnoExc.obj
 0004:00000334       ??_R0?AVEbusyExc@Iex@@@8   10021334     IexThrowErrnoExc.obj
 0004:00000354       ??_R0?AVEexistExc@Iex@@@8  10021354     IexThrowErrnoExc.obj
 0004:00000378       ??_R0?AVExdevExc@Iex@@@8   10021378     IexThrowErrnoExc.obj
 0004:00000398       ??_R0?AVEnodevExc@Iex@@@8  10021398     IexThrowErrnoExc.obj
 0004:000003bc       ??_R0?AVEnotdirExc@Iex@@@8 100213bc     IexThrowErrnoExc.obj
 0004:000003e0       ??_R0?AVEisdirExc@Iex@@@8  100213e0     IexThrowErrnoExc.obj
 0004:00000404       ??_R0?AVEinvalExc@Iex@@@8  10021404     IexThrowErrnoExc.obj
 0004:00000428       ??_R0?AVEnfileExc@Iex@@@8  10021428     IexThrowErrnoExc.obj
 0004:0000044c       ??_R0?AVEmfileExc@Iex@@@8  1002144c     IexThrowErrnoExc.obj
 0004:00000470       ??_R0?AVEnottyExc@Iex@@@8  10021470     IexThrowErrnoExc.obj
 0004:00000494       ??_R0?AVEfbigExc@Iex@@@8   10021494     IexThrowErrnoExc.obj
 0004:000004b4       ??_R0?AVEnospcExc@Iex@@@8  100214b4     IexThrowErrnoExc.obj
 0004:000004d8       ??_R0?AVEspipeExc@Iex@@@8  100214d8     IexThrowErrnoExc.obj
 0004:000004fc       ??_R0?AVErofsExc@Iex@@@8   100214fc     IexThrowErrnoExc.obj
 0004:0000051c       ??_R0?AVEmlinkExc@Iex@@@8  1002151c     IexThrowErrnoExc.obj
 0004:00000540       ??_R0?AVEpipeExc@Iex@@@8   10021540     IexThrowErrnoExc.obj
 0004:00000560       ??_R0?AVEdomExc@Iex@@@8    10021560     IexThrowErrnoExc.obj
 0004:00000580       ??_R0?AVErangeExc@Iex@@@8  10021580     IexThrowErrnoExc.obj
 0004:000005a4       ??_R0?AVEdeadlkExc@Iex@@@8 100215a4     IexThrowErrnoExc.obj
 0004:000005c8       ??_R0?AVEnolckExc@Iex@@@8  100215c8     IexThrowErrnoExc.obj
 0004:000005ec       ??_R0?AVEnametoolongExc@Iex@@@8 100215ec     IexThrowErrnoExc.obj
 0004:00000614       ??_R0?AVEilseqExc@Iex@@@8  10021614     IexThrowErrnoExc.obj
 0004:00000638       ??_R0?AVEnosysExc@Iex@@@8  10021638     IexThrowErrnoExc.obj
 0004:0000065c       ??_R0?AVEnotemptyExc@Iex@@@8 1002165c     IexThrowErrnoExc.obj
 0004:00000684       ??_R0?AVtype_info@@@8      10021684     MSVCRTD:ti_inst.obj
 0004:000006a0       ___security_cookie         100216a0     MSVCRTD:gs_cookie.obj
 0004:000006a4       ___security_cookie_complement 100216a4     MSVCRTD:gs_cookie.obj
 0004:000006c0       ?_RTC_ErrorLevels@@3PAHA   100216c0     MSVCRTD:error.obj
 0004:000006f4       ___native_dllmain_reason   100216f4     MSVCRTD:natstart.obj
 0004:000006f8       ___native_vcclrit_reason   100216f8     MSVCRTD:natstart.obj
 0004:00000838       ?currentStackTracer@?A0x883d44e9@Iex@@3P6A?AV?$basic_string@DU?$char_traits@D@std@@V?$allocator@D@2@@std@@XZA 10021838     IexBaseExc.obj
 0004:00000850       ?wsprintffp@@3P6AHPADPBDZZA 10021850     MSVCRTD:error.obj
 0004:00000c1c       ?__type_info_root_node@@3U__type_info_node@@A 10021c1c     MSVCRTD:tncleanup.obj
 0004:00000c34       __adjust_fdiv              10021c34     <common>
 0004:00000c40       ___native_startup_state    10021c40     <common>
 0004:00000c50       ___native_startup_lock     10021c50     <common>
 0004:00000c54       ___onexitend               10021c54     <common>
 0004:00000c64       ___onexitbegin             10021c64     <common>
 0004:00000c68       ___dyn_tls_init_callback   10021c68     <common>
 0005:00000000       __IMPORT_DESCRIPTOR_MSVCP80D 10022000     msvcprtd:MSVCP80D.dll
 0005:00000014       __IMPORT_DESCRIPTOR_MSVCR80D 10022014     MSVCRTD:MSVCR80D.dll
 0005:00000028       __IMPORT_DESCRIPTOR_KERNEL32 10022028     kernel32:KERNEL32.dll
 0005:0000003c       __NULL_IMPORT_DESCRIPTOR   1002203c     msvcprtd:MSVCP80D.dll
 0005:00000220       __imp__Sleep@4             10022220     kernel32:KERNEL32.dll
 0005:00000224       __imp__InterlockedCompareExchange@12 10022224     kernel32:KERNEL32.dll
 0005:00000228       __imp__RaiseException@16   10022228     kernel32:KERNEL32.dll
 0005:0000022c       __imp__DebugBreak@0        1002222c     kernel32:KERNEL32.dll
 0005:00000230       __imp__WideCharToMultiByte@32 10022230     kernel32:KERNEL32.dll
 0005:00000234       __imp__IsDebuggerPresent@0 10022234     kernel32:KERNEL32.dll
 0005:00000238       __imp__MultiByteToWideChar@24 10022238     kernel32:KERNEL32.dll
 0005:0000023c       __imp__lstrlenA@4          1002223c     kernel32:KERNEL32.dll
 0005:00000240       __imp__GetProcAddress@8    10022240     kernel32:KERNEL32.dll
 0005:00000244       __imp__LoadLibraryA@4      10022244     kernel32:KERNEL32.dll
 0005:00000248       __imp__TerminateProcess@8  10022248     kernel32:KERNEL32.dll
 0005:0000024c       __imp__GetCurrentProcess@0 1002224c     kernel32:KERNEL32.dll
 0005:00000250       __imp__FreeLibrary@4       10022250     kernel32:KERNEL32.dll
 0005:00000254       __imp__VirtualQuery@12     10022254     kernel32:KERNEL32.dll
 0005:00000258       __imp__GetModuleFileNameW@12 10022258     kernel32:KERNEL32.dll
 0005:0000025c       __imp__GetProcessHeap@0    1002225c     kernel32:KERNEL32.dll
 0005:00000260       __imp__HeapAlloc@12        10022260     kernel32:KERNEL32.dll
 0005:00000264       __imp__HeapFree@12         10022264     kernel32:KERNEL32.dll
 0005:00000268       __imp__DisableThreadLibraryCalls@4 10022268     kernel32:KERNEL32.dll
 0005:0000026c       __imp__FatalAppExitA@8     1002226c     kernel32:KERNEL32.dll
 0005:00000270       __imp__GetSystemTimeAsFileTime@4 10022270     kernel32:KERNEL32.dll
 0005:00000274       __imp__GetCurrentProcessId@0 10022274     kernel32:KERNEL32.dll
 0005:00000278       __imp__GetCurrentThreadId@0 10022278     kernel32:KERNEL32.dll
 0005:0000027c       __imp__GetTickCount@0      1002227c     kernel32:KERNEL32.dll
 0005:00000280       __imp__QueryPerformanceCounter@4 10022280     kernel32:KERNEL32.dll
 0005:00000284       __imp__SetUnhandledExceptionFilter@4 10022284     kernel32:KERNEL32.dll
 0005:00000288       __imp__UnhandledExceptionFilter@4 10022288     kernel32:KERNEL32.dll
 0005:0000028c       __imp__InterlockedExchange@8 1002228c     kernel32:KERNEL32.dll
 0005:00000290       \177KERNEL32_NULL_THUNK_DATA 10022290     kernel32:KERNEL32.dll
 0005:000002d0       __imp_??0_Container_base@std@@QAE@ABV01@@Z 100222d0     msvcprtd:MSVCP80D.dll
 0005:000002d4       __imp_??0_String_base@std@@QAE@ABV01@@Z 100222d4     msvcprtd:MSVCP80D.dll
 0005:000002d8       __imp_??0?$_String_val@DV?$allocator@D@std@@@std@@QAE@ABV01@@Z 100222d8     msvcprtd:MSVCP80D.dll
 0005:000002dc       __imp_?find@?$basic_string@DU?$char_traits@D@std@@V?$allocator@D@2@@std@@QBEIPBDI@Z 100222dc     msvcprtd:MSVCP80D.dll
 0005:000002e0       __imp_?replace@?$basic_string@DU?$char_traits@D@std@@V?$allocator@D@2@@std@@QAEAAV12@IIPBDI@Z 100222e0     msvcprtd:MSVCP80D.dll
 0005:000002e4       __imp_?append@?$basic_string@DU?$char_traits@D@std@@V?$allocator@D@2@@std@@QAEAAV12@ABV12@@Z 100222e4     msvcprtd:MSVCP80D.dll
 0005:000002e8       __imp_?assign@?$basic_string@DU?$char_traits@D@std@@V?$allocator@D@2@@std@@QAEAAV12@ABV12@@Z 100222e8     msvcprtd:MSVCP80D.dll
 0005:000002ec       __imp_??1?$basic_string@DU?$char_traits@D@std@@V?$allocator@D@2@@std@@QAE@XZ 100222ec     msvcprtd:MSVCP80D.dll
 0005:000002f0       __imp_?c_str@?$basic_string@DU?$char_traits@D@std@@V?$allocator@D@2@@std@@QBEPBDXZ 100222f0     msvcprtd:MSVCP80D.dll
 0005:000002f4       __imp_?str@?$basic_stringstream@DU?$char_traits@D@std@@V?$allocator@D@2@@std@@QBE?AV?$basic_string@DU?$char_traits@D@std@@V?$allocator@D@2@@2@XZ 100222f4     msvcprtd:MSVCP80D.dll
 0005:000002f8       __imp_??0?$basic_string@DU?$char_traits@D@std@@V?$allocator@D@2@@std@@QAE@PBD@Z 100222f8     msvcprtd:MSVCP80D.dll
 0005:000002fc       __imp_??0?$basic_string@DU?$char_traits@D@std@@V?$allocator@D@2@@std@@QAE@ABV01@@Z 100222fc     msvcprtd:MSVCP80D.dll
 0005:00000300       \177MSVCP80D_NULL_THUNK_DATA 10022300     msvcprtd:MSVCP80D.dll
 0005:00000334       __imp___onexit             10022334     MSVCRTD:MSVCR80D.dll
 0005:00000338       __imp___except_handler4_common 10022338     MSVCRTD:MSVCR80D.dll
 0005:0000033c       __imp___lock               1002233c     MSVCRTD:MSVCR80D.dll
 0005:00000340       __imp____dllonexit         10022340     MSVCRTD:MSVCR80D.dll
 0005:00000344       __imp___unlock             10022344     MSVCRTD:MSVCR80D.dll
 0005:00000348       __imp____clean_type_info_names_internal 10022348     MSVCRTD:MSVCR80D.dll
 0005:0000034c       __imp___crt_debugger_hook  1002234c     MSVCRTD:MSVCR80D.dll
 0005:00000350       __imp_?terminate@@YAXXZ    10022350     MSVCRTD:MSVCR80D.dll
 0005:00000354       __imp____CppXcptFilter     10022354     MSVCRTD:MSVCR80D.dll
 0005:00000358       __imp___adjust_fdiv        10022358     MSVCRTD:MSVCR80D.dll
 0005:0000035c       __imp___amsg_exit          1002235c     MSVCRTD:MSVCR80D.dll
 0005:00000360       __imp___initterm_e         10022360     MSVCRTD:MSVCR80D.dll
 0005:00000364       __imp___initterm           10022364     MSVCRTD:MSVCR80D.dll
 0005:00000368       __imp___CrtSetCheckCount   10022368     MSVCRTD:MSVCR80D.dll
 0005:0000036c       __imp___decode_pointer     1002236c     MSVCRTD:MSVCR80D.dll
 0005:00000370       __imp___free_dbg           10022370     MSVCRTD:MSVCR80D.dll
 0005:00000374       __imp___encoded_null       10022374     MSVCRTD:MSVCR80D.dll
 0005:00000378       __imp___malloc_dbg         10022378     MSVCRTD:MSVCR80D.dll
 0005:0000037c       __imp___encode_pointer     1002237c     MSVCRTD:MSVCR80D.dll
 0005:00000380       __imp___CRT_RTC_INITW      10022380     MSVCRTD:MSVCR80D.dll
 0005:00000384       __imp___errno              10022384     MSVCRTD:MSVCR80D.dll
 0005:00000388       __imp_??0exception@std@@QAE@ABV01@@Z 10022388     MSVCRTD:MSVCR80D.dll
 0005:0000038c       __imp___CxxThrowException@8 1002238c     MSVCRTD:MSVCR80D.dll
 0005:00000390       __imp__strerror            10022390     MSVCRTD:MSVCR80D.dll
 0005:00000394       __imp__strlen              10022394     MSVCRTD:MSVCR80D.dll
 0005:00000398       __imp____CxxFrameHandler3  10022398     MSVCRTD:MSVCR80D.dll
 0005:0000039c       __imp_??1exception@std@@UAE@XZ 1002239c     MSVCRTD:MSVCR80D.dll
 0005:000003a0       __imp_??3@YAXPAX@Z         100223a0     MSVCRTD:MSVCR80D.dll
 0005:000003a4       __imp_??0exception@std@@QAE@XZ 100223a4     MSVCRTD:MSVCR80D.dll
 0005:000003a8       __imp_?_type_info_dtor_internal_method@type_info@@QAEXXZ 100223a8     MSVCRTD:MSVCR80D.dll
 0005:000003ac       \177MSVCR80D_NULL_THUNK_DATA 100223ac     MSVCRTD:MSVCR80D.dll

 entry point at        0002:00000352

